 getcaps002

 Timestamp is 926a3cfc (reproducible build file hash)

 Preferred load address is 0000000180000000

 Start         Length     Name                   Class
 0001:00000000 00004160H .text$mn                CODE
 0001:00004160 00000036H .text$mn$00             CODE
 0001:00004196 00000092H .text$x                 CODE
 0002:00000000 000001c8H .idata$5                DATA
 0002:000001c8 00000038H .00cfg                  DATA
 0002:00000200 00000008H .CRT$XCA                DATA
 0002:00000208 00000008H .CRT$XCZ                DATA
 0002:00000210 00000008H .CRT$XIA                DATA
 0002:00000218 00000008H .CRT$XIC                DATA
 0002:00000220 00000008H .CRT$XIZ                DATA
 0002:00000228 00000008H .CRT$XLA                DATA
 0002:00000230 00000008H .CRT$XLZ                DATA
 0002:00000238 00000008H .CRT$XPA                DATA
 0002:00000240 00000008H .CRT$XPZ                DATA
 0002:00000248 00000008H .CRT$XTA                DATA
 0002:00000250 00000010H .CRT$XTZ                DATA
 0002:00000258 00000000H .gehcont$y              DATA
 0002:00000258 00000000H .gfids$y                DATA
 0002:00000260 000025a0H .rdata                  DATA
 0002:00002800 00000000H .rdata$CastGuardVftablesA DATA
 0002:00002800 00000000H .rdata$CastGuardVftablesC DATA
 0002:00002800 00000028H .rdata$T                DATA
 0002:00002828 000000bcH .rdata$voltmd           DATA
 0002:000028e4 0000031cH .rdata$zzzdbg           DATA
 0002:00002c00 00000008H .rtc$IAA                DATA
 0002:00002c08 00000008H .rtc$IZZ                DATA
 0002:00002c10 00000008H .rtc$TAA                DATA
 0002:00002c18 00000008H .rtc$TZZ                DATA
 0002:00002c20 00000004H .tls                    DATA
 0002:00002c24 00000004H .tls$                   DATA
 0002:00002c28 00000008H .tls$ZZZ                DATA
 0002:00002c30 00000380H .xdata                  DATA
 0002:00002fb0 00000398H .edata                  DATA
 0002:00003348 0000008cH .idata$2                DATA
 0002:000033d4 00000014H .idata$3                DATA
 0002:000033e8 000001c8H .idata$4                DATA
 0002:000035b0 00000486H .idata$6                DATA
 0003:00000000 00000080H .data                   DATA
 0003:00000080 0001b238H .bss                    DATA
 0004:00000000 00000414H .pdata                  DATA

  Address         Publics by Value              Rva+Base               Lib:Object

 0000:00000000       __AbsoluteZero             0000000000000000     <absolute>
 0000:00000000       ___safe_se_handler_count   0000000000000000     <absolute>
 0000:00000000       ___safe_se_handler_table   0000000000000000     <absolute>
 0000:00000000       __arm64x_extra_rfe_table   0000000000000000     <absolute>
 0000:00000000       __arm64x_extra_rfe_table_size 0000000000000000     <absolute>
 0000:00000000       __arm64x_native_entrypoint 0000000000000000     <absolute>
 0000:00000000       __arm64x_redirection_metadata 0000000000000000     <absolute>
 0000:00000000       __arm64x_redirection_metadata_count 0000000000000000     <absolute>
 0000:00000000       __dynamic_value_reloc_table 0000000000000000     <absolute>
 0000:00000000       __enclave_config           0000000000000000     <absolute>
 0000:00000000       __guard_check_icall_a64n_fptr 0000000000000000     <absolute>
 0000:00000000       __guard_eh_cont_count      0000000000000000     <absolute>
 0000:00000000       __guard_eh_cont_table      0000000000000000     <absolute>
 0000:00000000       __guard_fids_count         0000000000000000     <absolute>
 0000:00000000       __guard_fids_table         0000000000000000     <absolute>
 0000:00000000       __guard_iat_count          0000000000000000     <absolute>
 0000:00000000       __guard_iat_table          0000000000000000     <absolute>
 0000:00000000       __guard_longjmp_count      0000000000000000     <absolute>
 0000:00000000       __guard_longjmp_table      0000000000000000     <absolute>
 0000:00000000       __hybrid_auxiliary_iat     0000000000000000     <absolute>
 0000:00000000       __hybrid_auxiliary_iat_copy 0000000000000000     <absolute>
 0000:00000000       __hybrid_code_map          0000000000000000     <absolute>
 0000:00000000       __hybrid_code_map_count    0000000000000000     <absolute>
 0000:00000000       __x64_code_ranges_to_entry_points 0000000000000000     <absolute>
 0000:00000000       __x64_code_ranges_to_entry_points_count 0000000000000000     <absolute>
 0000:00000100       __guard_flags              0000000000000100     <absolute>
 0000:00000000       __ImageBase                0000000180000000     <linker-defined>
 0001:00000000       ?NewObject@JNIEnv_@@QEAAPEAV_jobject@@PEAV_jclass@@PEAU_jmethodID@@ZZ 0000000180001000 f i libgetcaps002.obj
 0001:00000028       ?SetEventNotificationMode@_jvmtiEnv@@QEAA?AW4jvmtiError@@W4jvmtiEventMode@@W4jvmtiEvent@@PEAV_jobject@@ZZ 0000000180001028 f i libgetcaps002.obj
 0001:00000034       ?TranslateError@@YAPEBDW4jvmtiError@@@Z 0000000180001034 f   libgetcaps002.obj
 0001:000002ec       ?nsk_jni_check_exception@@YAHPEAUJNIEnv_@@QEBDH@Z 00000001800012ec f   libgetcaps002.obj
 0001:00000430       ?nsk_jni_lverify@@YAHHPEAUJNIEnv_@@HQEBDH1ZZ 0000000180001430 f   libgetcaps002.obj
 0001:000004d0       Agent_Initialize           00000001800014d0 f   libgetcaps002.obj
 0001:00000738       Agent_OnAttach             0000000180001738 f   libgetcaps002.obj
 0001:00000738       Agent_OnLoad               0000000180001738 f   libgetcaps002.obj
 0001:00000740       Java_nsk_jvmti_unit_FollowReferences_FollowRefObjects_addRefToVerify 0000000180001740 f   libgetcaps002.obj
 0001:00000918       Java_nsk_jvmti_unit_FollowReferences_FollowRefObjects_getTag 0000000180001918 f   libgetcaps002.obj
 0001:000009d8       Java_nsk_jvmti_unit_FollowReferences_FollowRefObjects_resetRefsToVerify 00000001800019d8 f   libgetcaps002.obj
 0001:000009e0       Java_nsk_jvmti_unit_FollowReferences_FollowRefObjects_resetTags 00000001800019e0 f   libgetcaps002.obj
 0001:00000a24       Java_nsk_jvmti_unit_FollowReferences_FollowRefObjects_setTag 0000000180001a24 f   libgetcaps002.obj
 0001:00000c7c       Java_nsk_share_jvmti_ArgumentHandler_getAgentOptionsString 0000000180001c7c f   libgetcaps002.obj
 0001:00000d2c       Java_nsk_share_jvmti_DebugeeClass_checkStatus 0000000180001d2c f   libgetcaps002.obj
 0001:00000db4       Java_nsk_share_jvmti_DebugeeClass_resetAgentData 0000000180001db4 f   libgetcaps002.obj
 0001:00000e14       Java_nsk_share_jvmti_RedefineAgent_agentStatus 0000000180001e14 f   libgetcaps002.obj
 0001:00000e20       Java_nsk_share_jvmti_RedefineAgent_isRedefined 0000000180001e20 f   libgetcaps002.obj
 0001:00000e2c       Java_nsk_share_jvmti_RedefineAgent_redefineAttempted 0000000180001e2c f   libgetcaps002.obj
 0001:00000e38       MA_checkStatus             0000000180001e38 f   libgetcaps002.obj
 0001:00000edc       __local_stdio_printf_options 0000000180001edc f i libgetcaps002.obj
 0001:00001144       callbackVMDeath            0000000180002144 f   libgetcaps002.obj
 0001:0000121c       callbackVMInit             000000018000221c f   libgetcaps002.obj
 0001:00001c48       exitOnError                0000000180002c48 f   libgetcaps002.obj
 0001:00001cfc       fprintf                    0000000180002cfc f i libgetcaps002.obj
 0001:00001d40       nsk_complain               0000000180002d40 f   libgetcaps002.obj
 0001:00001d6c       nsk_jvmti_createJVMTIEnv   0000000180002d6c f   libgetcaps002.obj
 0001:00001e9c       nsk_jvmti_enableEvents     0000000180002e9c f   libgetcaps002.obj
 0001:00001f70       nsk_jvmti_lverify          0000000180002f70 f   libgetcaps002.obj
 0001:00002060       nsk_jvmti_parseOptions     0000000180003060 f   libgetcaps002.obj
 0001:000022b0       nsk_jvmti_resetAgentData   00000001800032b0 f   libgetcaps002.obj
 0001:00002330       nsk_jvmti_resumeSync       0000000180003330 f   libgetcaps002.obj
 0001:000023d8       nsk_jvmti_setFailStatus    00000001800033d8 f   libgetcaps002.obj
 0001:00002414       nsk_jvmti_waitForSync      0000000180003414 f   libgetcaps002.obj
 0001:00002518       nsk_lcomplain              0000000180003518 f   libgetcaps002.obj
 0001:00002538       nsk_ldisplay               0000000180003538 f   libgetcaps002.obj
 0001:00002558       nsk_ltrace                 0000000180003558 f   libgetcaps002.obj
 0001:00002578       nsk_lvcomplain             0000000180003578 f   libgetcaps002.obj
 0001:00002730       nsk_lvdisplay              0000000180003730 f   libgetcaps002.obj
 0001:0000277c       nsk_lverify                000000018000377c f   libgetcaps002.obj
 0001:000027d8       nsk_lvtrace                00000001800037d8 f   libgetcaps002.obj
 0001:00002838       nsk_printf                 0000000180003838 f   libgetcaps002.obj
 0001:00002860       nsk_vprintf                0000000180003860 f   libgetcaps002.obj
 0001:00002d14       printf                     0000000180003d14 f i libgetcaps002.obj
 0001:0000323c       __raise_securityfailure    000000018000423c f   MSVCRT:gs_report.obj
 0001:00003270       __report_gsfailure         0000000180004270 f   MSVCRT:gs_report.obj
 0001:000034b0       __GSHandlerCheck           00000001800044b0 f   MSVCRT:gshandler.obj
 0001:000034d0       __GSHandlerCheckCommon     00000001800044d0 f   MSVCRT:gshandler.obj
 0001:00003540       __security_check_cookie    0000000180004540 f   MSVCRT:amdsecgs.obj
 0001:00003880       _DllMainCRTStartup         0000000180004880 f   MSVCRT:dll_dllmain.obj
 0001:000038c0       __scrt_acquire_startup_lock 00000001800048c0 f   MSVCRT:utility.obj
 0001:000038fc       __scrt_dllmain_after_initialize_c 00000001800048fc f   MSVCRT:utility.obj
 0001:00003930       __scrt_dllmain_before_initialize_c 0000000180004930 f   MSVCRT:utility.obj
 0001:00003948       __scrt_dllmain_crt_thread_attach 0000000180004948 f   MSVCRT:utility.obj
 0001:00003970       __scrt_dllmain_crt_thread_detach 0000000180004970 f   MSVCRT:utility.obj
 0001:00003988       __scrt_dllmain_exception_filter 0000000180004988 f   MSVCRT:utility.obj
 0001:000039e8       __scrt_dllmain_uninitialize_c 00000001800049e8 f   MSVCRT:utility.obj
 0001:00003a18       __scrt_dllmain_uninitialize_critical 0000000180004a18 f   MSVCRT:utility.obj
 0001:00003a2c       __scrt_initialize_crt      0000000180004a2c f   MSVCRT:utility.obj
 0001:00003a78       __scrt_initialize_onexit_tables 0000000180004a78 f   MSVCRT:utility.obj
 0001:00003b04       __scrt_is_nonwritable_in_current_image 0000000180004b04 f   MSVCRT:utility.obj
 0001:00003b9c       __scrt_release_startup_lock 0000000180004b9c f   MSVCRT:utility.obj
 0001:00003bc0       __scrt_uninitialize_crt    0000000180004bc0 f   MSVCRT:utility.obj
 0001:00003bec       _onexit                    0000000180004bec f   MSVCRT:utility.obj
 0001:00003c28       atexit                     0000000180004c28 f   MSVCRT:utility.obj
 0001:00003c40       __crt_debugger_hook        0000000180004c40 f   MSVCRT:utility_desktop.obj
 0001:00003c48       __scrt_fastfail            0000000180004c48 f   MSVCRT:utility_desktop.obj
 0001:00003d94       _guard_check_icall_nop     0000000180004d94 f i MSVCRT:guard_support.obj
 0001:00003d98       __security_init_cookie     0000000180004d98 f   MSVCRT:gs_support.obj
 0001:00003e44       DllMain                    0000000180004e44 f   MSVCRT:dll_dllmain_stub.obj
 0001:00003e68       ?__scrt_initialize_type_info@@YAXXZ 0000000180004e68 f   MSVCRT:tncleanup.obj
 0001:00003e78       ?__scrt_uninitialize_type_info@@YAXXZ 0000000180004e78 f   MSVCRT:tncleanup.obj
 0001:00003e84       __local_stdio_scanf_options 0000000180004e84 f i MSVCRT:default_local_stdio_options.obj
 0001:00003e8c       __scrt_initialize_default_local_stdio_options 0000000180004e8c f   MSVCRT:default_local_stdio_options.obj
 0001:00003ea8       __scrt_get_dyn_tls_init_callback 0000000180004ea8 f   MSVCRT:dyn_tls_init.obj
 0001:00003eb0       _RTC_Initialize            0000000180004eb0 f   MSVCRT:initsect.obj
 0001:00003eec       _RTC_Terminate             0000000180004eec f   MSVCRT:initsect.obj
 0001:00003f28       __isa_available_init       0000000180004f28 f   MSVCRT:cpu_disp.obj
 0001:000040d4       _get_startup_argv_mode     00000001800050d4 f   MSVCRT:argv_mode.obj
 0001:000040dc       __scrt_is_ucrt_dll_in_use  00000001800050dc f   MSVCRT:ucrt_detection.obj
 0001:000040f0       memcpy                     00000001800050f0 f   vcruntime:VCRUNTIME140.dll
 0001:000040f6       memset                     00000001800050f6 f   vcruntime:VCRUNTIME140.dll
 0001:000040fc       strchr                     00000001800050fc f   vcruntime:VCRUNTIME140.dll
 0001:00004102       __C_specific_handler       0000000180005102 f   vcruntime:VCRUNTIME140.dll
 0001:00004108       __std_type_info_destroy_list 0000000180005108 f   vcruntime:VCRUNTIME140.dll
 0001:0000410e       strcmp                     000000018000510e f   ucrt:api-ms-win-crt-string-l1-1-0.dll
 0001:00004114       strlen                     0000000180005114 f   ucrt:api-ms-win-crt-string-l1-1-0.dll
 0001:0000411a       _initterm                  000000018000511a f   ucrt:api-ms-win-crt-runtime-l1-1-0.dll
 0001:00004120       _initterm_e                0000000180005120 f   ucrt:api-ms-win-crt-runtime-l1-1-0.dll
 0001:00004126       _seh_filter_dll            0000000180005126 f   ucrt:api-ms-win-crt-runtime-l1-1-0.dll
 0001:0000412c       _configure_narrow_argv     000000018000512c f   ucrt:api-ms-win-crt-runtime-l1-1-0.dll
 0001:00004132       _initialize_narrow_environment 0000000180005132 f   ucrt:api-ms-win-crt-runtime-l1-1-0.dll
 0001:00004138       _initialize_onexit_table   0000000180005138 f   ucrt:api-ms-win-crt-runtime-l1-1-0.dll
 0001:0000413e       _register_onexit_function  000000018000513e f   ucrt:api-ms-win-crt-runtime-l1-1-0.dll
 0001:00004144       _execute_onexit_table      0000000180005144 f   ucrt:api-ms-win-crt-runtime-l1-1-0.dll
 0001:0000414a       _crt_atexit                000000018000514a f   ucrt:api-ms-win-crt-runtime-l1-1-0.dll
 0001:00004150       _cexit                     0000000180005150 f   ucrt:api-ms-win-crt-runtime-l1-1-0.dll
 0001:00004158       __acrt_initialize          0000000180005158 f   MSVCRT:ucrt_stubs.obj
 0001:00004158       __acrt_thread_attach       0000000180005158 f   MSVCRT:ucrt_stubs.obj
 0001:00004158       __acrt_thread_detach       0000000180005158 f   MSVCRT:ucrt_stubs.obj
 0001:00004158       __acrt_uninitialize        0000000180005158 f   MSVCRT:ucrt_stubs.obj
 0001:00004158       __acrt_uninitialize_critical 0000000180005158 f   MSVCRT:ucrt_stubs.obj
 0001:00004158       __scrt_stub_for_acrt_initialize 0000000180005158 f   MSVCRT:ucrt_stubs.obj
 0001:00004158       __scrt_stub_for_acrt_thread_attach 0000000180005158 f   MSVCRT:ucrt_stubs.obj
 0001:00004158       __scrt_stub_for_acrt_thread_detach 0000000180005158 f   MSVCRT:ucrt_stubs.obj
 0001:00004158       __scrt_stub_for_acrt_uninitialize 0000000180005158 f   MSVCRT:ucrt_stubs.obj
 0001:00004158       __scrt_stub_for_acrt_uninitialize_critical 0000000180005158 f   MSVCRT:ucrt_stubs.obj
 0001:00004158       __vcrt_initialize          0000000180005158 f   MSVCRT:ucrt_stubs.obj
 0001:00004158       __vcrt_thread_attach       0000000180005158 f   MSVCRT:ucrt_stubs.obj
 0001:00004158       __vcrt_thread_detach       0000000180005158 f   MSVCRT:ucrt_stubs.obj
 0001:00004158       __vcrt_uninitialize        0000000180005158 f   MSVCRT:ucrt_stubs.obj
 0001:00004158       __vcrt_uninitialize_critical 0000000180005158 f   MSVCRT:ucrt_stubs.obj
 0001:0000415c       __scrt_stub_for_is_c_termination_complete 000000018000515c f   MSVCRT:ucrt_stubs.obj
 0001:0000415c       _is_c_termination_complete 000000018000515c f   MSVCRT:ucrt_stubs.obj
 0001:00004170       _guard_dispatch_icall_nop  0000000180005170 f   MSVCRT:guard_dispatch.obj
 0001:00004190       _guard_xfg_dispatch_icall_nop 0000000180005190 f   MSVCRT:guard_xfg_dispatch.obj
 0002:00000000       __imp_RtlCaptureContext    0000000180006000     kernel32:KERNEL32.dll
 0002:00000008       __imp_RtlLookupFunctionEntry 0000000180006008     kernel32:KERNEL32.dll
 0002:00000010       __imp_RtlVirtualUnwind     0000000180006010     kernel32:KERNEL32.dll
 0002:00000018       __imp_UnhandledExceptionFilter 0000000180006018     kernel32:KERNEL32.dll
 0002:00000020       __imp_SetUnhandledExceptionFilter 0000000180006020     kernel32:KERNEL32.dll
 0002:00000028       __imp_GetCurrentProcess    0000000180006028     kernel32:KERNEL32.dll
 0002:00000030       __imp_TerminateProcess     0000000180006030     kernel32:KERNEL32.dll
 0002:00000038       __imp_IsProcessorFeaturePresent 0000000180006038     kernel32:KERNEL32.dll
 0002:00000040       __imp_CloseHandle          0000000180006040     kernel32:KERNEL32.dll
 0002:00000048       __imp_InitializeCriticalSectionAndSpinCount 0000000180006048     kernel32:KERNEL32.dll
 0002:00000050       __imp_DeleteCriticalSection 0000000180006050     kernel32:KERNEL32.dll
 0002:00000058       __imp_CreateEventW         0000000180006058     kernel32:KERNEL32.dll
 0002:00000060       __imp_GetModuleHandleW     0000000180006060     kernel32:KERNEL32.dll
 0002:00000068       __imp_GetProcAddress       0000000180006068     kernel32:KERNEL32.dll
 0002:00000070       __imp_IsDebuggerPresent    0000000180006070     kernel32:KERNEL32.dll
 0002:00000078       __imp_QueryPerformanceCounter 0000000180006078     kernel32:KERNEL32.dll
 0002:00000080       __imp_GetCurrentProcessId  0000000180006080     kernel32:KERNEL32.dll
 0002:00000088       __imp_GetCurrentThreadId   0000000180006088     kernel32:KERNEL32.dll
 0002:00000090       __imp_GetSystemTimeAsFileTime 0000000180006090     kernel32:KERNEL32.dll
 0002:00000098       __imp_DisableThreadLibraryCalls 0000000180006098     kernel32:KERNEL32.dll
 0002:000000a0       __imp_InitializeSListHead  00000001800060a0     kernel32:KERNEL32.dll
 0002:000000a8       \177KERNEL32_NULL_THUNK_DATA 00000001800060a8     kernel32:KERNEL32.dll
 0002:000000b0       __imp_memcpy               00000001800060b0     vcruntime:VCRUNTIME140.dll
 0002:000000b8       __imp_memset               00000001800060b8     vcruntime:VCRUNTIME140.dll
 0002:000000c0       __imp_strchr               00000001800060c0     vcruntime:VCRUNTIME140.dll
 0002:000000c8       __imp___C_specific_handler 00000001800060c8     vcruntime:VCRUNTIME140.dll
 0002:000000d0       __imp___std_type_info_destroy_list 00000001800060d0     vcruntime:VCRUNTIME140.dll
 0002:000000d8       \177VCRUNTIME140_NULL_THUNK_DATA 00000001800060d8     vcruntime:VCRUNTIME140.dll
 0002:000000e0       __imp_strtol               00000001800060e0     ucrt:api-ms-win-crt-convert-l1-1-0.dll
 0002:000000e8       \177api-ms-win-crt-convert-l1-1-0_NULL_THUNK_DATA 00000001800060e8     ucrt:api-ms-win-crt-convert-l1-1-0.dll
 0002:000000f0       __imp_malloc               00000001800060f0     ucrt:api-ms-win-crt-heap-l1-1-0.dll
 0002:000000f8       __imp_free                 00000001800060f8     ucrt:api-ms-win-crt-heap-l1-1-0.dll
 0002:00000100       \177api-ms-win-crt-heap-l1-1-0_NULL_THUNK_DATA 0000000180006100     ucrt:api-ms-win-crt-heap-l1-1-0.dll
 0002:00000108       __imp__errno               0000000180006108     ucrt:api-ms-win-crt-runtime-l1-1-0.dll
 0002:00000110       __imp_exit                 0000000180006110     ucrt:api-ms-win-crt-runtime-l1-1-0.dll
 0002:00000118       __imp__cexit               0000000180006118     ucrt:api-ms-win-crt-runtime-l1-1-0.dll
 0002:00000120       __imp__crt_atexit          0000000180006120     ucrt:api-ms-win-crt-runtime-l1-1-0.dll
 0002:00000128       __imp__execute_onexit_table 0000000180006128     ucrt:api-ms-win-crt-runtime-l1-1-0.dll
 0002:00000130       __imp__register_onexit_function 0000000180006130     ucrt:api-ms-win-crt-runtime-l1-1-0.dll
 0002:00000138       __imp__initialize_onexit_table 0000000180006138     ucrt:api-ms-win-crt-runtime-l1-1-0.dll
 0002:00000140       __imp__initialize_narrow_environment 0000000180006140     ucrt:api-ms-win-crt-runtime-l1-1-0.dll
 0002:00000148       __imp__configure_narrow_argv 0000000180006148     ucrt:api-ms-win-crt-runtime-l1-1-0.dll
 0002:00000150       __imp__seh_filter_dll      0000000180006150     ucrt:api-ms-win-crt-runtime-l1-1-0.dll
 0002:00000158       __imp__initterm_e          0000000180006158     ucrt:api-ms-win-crt-runtime-l1-1-0.dll
 0002:00000160       __imp__initterm            0000000180006160     ucrt:api-ms-win-crt-runtime-l1-1-0.dll
 0002:00000168       \177api-ms-win-crt-runtime-l1-1-0_NULL_THUNK_DATA 0000000180006168     ucrt:api-ms-win-crt-runtime-l1-1-0.dll
 0002:00000170       __imp___acrt_iob_func      0000000180006170     ucrt:api-ms-win-crt-stdio-l1-1-0.dll
 0002:00000178       __imp_fflush               0000000180006178     ucrt:api-ms-win-crt-stdio-l1-1-0.dll
 0002:00000180       __imp___stdio_common_vsprintf 0000000180006180     ucrt:api-ms-win-crt-stdio-l1-1-0.dll
 0002:00000188       __imp___stdio_common_vfprintf 0000000180006188     ucrt:api-ms-win-crt-stdio-l1-1-0.dll
 0002:00000190       \177api-ms-win-crt-stdio-l1-1-0_NULL_THUNK_DATA 0000000180006190     ucrt:api-ms-win-crt-stdio-l1-1-0.dll
 0002:00000198       __imp_strcmp               0000000180006198     ucrt:api-ms-win-crt-string-l1-1-0.dll
 0002:000001a0       __imp__strdup              00000001800061a0     ucrt:api-ms-win-crt-string-l1-1-0.dll
 0002:000001a0       __imp_strdup               00000001800061a0     ucrt:api-ms-win-crt-string-l1-1-0.dll
 0002:000001a8       __imp_strlen               00000001800061a8     ucrt:api-ms-win-crt-string-l1-1-0.dll
 0002:000001b0       __imp_strpbrk              00000001800061b0     ucrt:api-ms-win-crt-string-l1-1-0.dll
 0002:000001b8       __imp_strncpy              00000001800061b8     ucrt:api-ms-win-crt-string-l1-1-0.dll
 0002:000001c0       \177api-ms-win-crt-string-l1-1-0_NULL_THUNK_DATA 00000001800061c0     ucrt:api-ms-win-crt-string-l1-1-0.dll
 0002:000001c8       __guard_check_icall_fptr   00000001800061c8     MSVCRT:guard_support.obj
 0002:000001d0       __guard_xfg_check_icall_fptr 00000001800061d0     MSVCRT:guard_support.obj
 0002:000001d8       __guard_dispatch_icall_fptr 00000001800061d8     MSVCRT:guard_support.obj
 0002:000001e0       __guard_xfg_dispatch_icall_fptr 00000001800061e0     MSVCRT:guard_support.obj
 0002:000001e8       __guard_xfg_table_dispatch_icall_fptr 00000001800061e8     MSVCRT:guard_support.obj
 0002:000001f0       __castguard_check_failure_os_handled_fptr 00000001800061f0     MSVCRT:guard_support.obj
 0002:000001f8       __guard_memcpy_fptr        00000001800061f8     vcruntime:softmemtag.obj
 0002:00000200       __xc_a                     0000000180006200     MSVCRT:initializers.obj
 0002:00000208       __xc_z                     0000000180006208     MSVCRT:initializers.obj
 0002:00000210       __xi_a                     0000000180006210     MSVCRT:initializers.obj
 0002:00000220       __xi_z                     0000000180006220     MSVCRT:initializers.obj
 0002:00000228       __xl_a                     0000000180006228     MSVCRT:tlssup.obj
 0002:00000230       __xl_z                     0000000180006230     MSVCRT:tlssup.obj
 0002:00000238       __xp_a                     0000000180006238     MSVCRT:initializers.obj
 0002:00000240       __xp_z                     0000000180006240     MSVCRT:initializers.obj
 0002:00000248       __xt_a                     0000000180006248     MSVCRT:initializers.obj
 0002:00000250       __xt_z                     0000000180006250     MSVCRT:initializers.obj
 0002:00000260       g_refKindStr               0000000180006260     libgetcaps002.obj
 0002:00000410       ??_C@_09BPLDFGCI@unknown_0@ 0000000180006410     libgetcaps002.obj
 0002:00000420       ??_C@_0BL@FPNMECJD@JVMTI_HEAP_REFERENCE_CLASS@ 0000000180006420     libgetcaps002.obj
 0002:00000440       ??_C@_0BL@FKGKKLNM@JVMTI_HEAP_REFERENCE_FIELD@ 0000000180006440     libgetcaps002.obj
 0002:00000460       ??_C@_0CD@CAEHCFJF@JVMTI_HEAP_REFERENCE_ARRAY_ELEM@ 0000000180006460     libgetcaps002.obj
 0002:00000488       ??_C@_0CC@DNEBMCNK@JVMTI_HEAP_REFERENCE_CLASS_LOAD@ 0000000180006488     libgetcaps002.obj
 0002:000004b0       ??_C@_0BN@CJMIPEBB@JVMTI_HEAP_REFERENCE_SIGNERS@ 00000001800064b0     libgetcaps002.obj
 0002:000004d0       ??_C@_0CH@HBOIDPEB@JVMTI_HEAP_REFERENCE_PROTECTION@ 00000001800064d0     libgetcaps002.obj
 0002:000004f8       ??_C@_0BP@MDKGDGKL@JVMTI_HEAP_REFERENCE_INTERFACE@ 00000001800064f8     libgetcaps002.obj
 0002:00000518       ??_C@_0CC@JJMIHNJH@JVMTI_HEAP_REFERENCE_STATIC_FIE@ 0000000180006518     libgetcaps002.obj
 0002:00000540       ??_C@_0CD@IDHEEGID@JVMTI_HEAP_REFERENCE_CONSTANT_P@ 0000000180006540     libgetcaps002.obj
 0002:00000568       ??_C@_0CA@EFFCHNG@JVMTI_HEAP_REFERENCE_SUPERCLASS@ 0000000180006568     libgetcaps002.obj
 0002:00000588       ??_C@_0L@PCDFHGCJ@unknown_11@ 0000000180006588     libgetcaps002.obj
 0002:00000598       ??_C@_0L@NJBICFOK@unknown_12@ 0000000180006598     libgetcaps002.obj
 0002:000005a8       ??_C@_0L@MAADBEKL@unknown_13@ 00000001800065a8     libgetcaps002.obj
 0002:000005b8       ??_C@_0L@IPECICGM@unknown_14@ 00000001800065b8     libgetcaps002.obj
 0002:000005c8       ??_C@_0L@JGFJLDCN@unknown_15@ 00000001800065c8     libgetcaps002.obj
 0002:000005d8       ??_C@_0L@LNHEOAOO@unknown_16@ 00000001800065d8     libgetcaps002.obj
 0002:000005e8       ??_C@_0L@KEGPNBKP@unknown_17@ 00000001800065e8     libgetcaps002.obj
 0002:000005f8       ??_C@_0L@CDPHMNGA@unknown_18@ 00000001800065f8     libgetcaps002.obj
 0002:00000608       ??_C@_0L@DKOMPMCB@unknown_19@ 0000000180006608     libgetcaps002.obj
 0002:00000618       ??_C@_0L@OJGIPJDB@unknown_20@ 0000000180006618     libgetcaps002.obj
 0002:00000628       ??_C@_0CA@KAOFNDEM@JVMTI_HEAP_REFERENCE_JNI_GLOBAL@ 0000000180006628     libgetcaps002.obj
 0002:00000648       ??_C@_0CC@HPFAJBK@JVMTI_HEAP_REFERENCE_SYSTEM_CLA@ 0000000180006648     libgetcaps002.obj
 0002:00000670       ??_C@_0BN@FDEGFOHC@JVMTI_HEAP_REFERENCE_MONITOR@ 0000000180006670     libgetcaps002.obj
 0002:00000690       ??_C@_0CB@HKIBCMAJ@JVMTI_HEAP_REFERENCE_STACK_LOCA@ 0000000180006690     libgetcaps002.obj
 0002:000006b8       ??_C@_0BP@EAACMMOE@JVMTI_HEAP_REFERENCE_JNI_LOCAL@ 00000001800066b8     libgetcaps002.obj
 0002:000006d8       ??_C@_0BM@IJDEOGOE@JVMTI_HEAP_REFERENCE_THREAD@ 00000001800066d8     libgetcaps002.obj
 0002:000006f8       ??_C@_0BL@EDGPPKC@JVMTI_HEAP_REFERENCE_OTHER@ 00000001800066f8     libgetcaps002.obj
 0002:00000714       ??_C@_04BCJPDBDA@Code@     0000000180006714     libgetcaps002.obj
 0002:00000720       ??_C@_0BA@OCLMCFKC@LineNumberTable@ 0000000180006720     libgetcaps002.obj
 0002:00000730       ??_C@_0BD@CPAEPILC@LocalVariableTable@ 0000000180006730     libgetcaps002.obj
 0002:00000748       ??_C@_0BH@NMBDNHBD@LocalVariableTypeTable@ 0000000180006748     libgetcaps002.obj
 0002:00000760       ??_C@_0O@HIHEEDNJ@StackMapTable@ 0000000180006760     libgetcaps002.obj
 0002:00000770       ??_C@_0L@HCDIAMJG@?9?5?$CFs?0?5?$CFd?3?5@ 0000000180006770     libgetcaps002.obj
 0002:00000780       ??_C@_0JI@HLPECLFI@?$CD?5?4?4?4?6?$CD?5ERROR?3?5too?5many?5complai@ 0000000180006780     libgetcaps002.obj
 0002:00000820       ??_C@_0ED@JNEKCCOB@The?5following?5fake?5exception?5st@ 0000000180006820     libgetcaps002.obj
 0002:00000868       ??_C@_0CN@FCNMDFBH@nsk?4share?4Fake_Exception_for_RU@ 0000000180006868     libgetcaps002.obj
 0002:00000898       ??_C@_08PGFFNAEI@?$CI?$CFs?3?$CFd?$CJ?5@ 0000000180006898     libgetcaps002.obj
 0002:000008a8       ??_C@_0DP@IENMAEGI@s?2test?2hotspot?2jtreg?2vmTestbase@ 00000001800068a8     libgetcaps002.obj
 0002:000008e8       ??_C@_0BL@NDJLFFJB@?7at?5nsk_lvcomplain?$CI?$CFs?3?$CFd?$CJ?6@ 00000001800068e8     libgetcaps002.obj
 0002:00000908       ??_C@_0BC@JOOKAFKF@?$CD?5ERROR?3?5?$CFs?0?5?$CFd?3?5@ 0000000180006908     libgetcaps002.obj
 0002:00000920       ??_C@_09KJEAHMEH@?$CD?5ERROR?3?5@ 0000000180006920     libgetcaps002.obj
 0002:0000092c       ??_C@_02GPIOPFAK@?$DO?$DO@ 000000018000692c     libgetcaps002.obj
 0002:00000930       ??_C@_02FODMEDOG@?$DM?$DM@ 0000000180006930     libgetcaps002.obj
 0002:00000934       ??_C@_02DJGKEECL@?4?4@     0000000180006934     libgetcaps002.obj
 0002:00000938       ??_C@_0O@CJPGJOAF@?9?5?$CFs?0?5?$CFd?3?5?$CFs?5@ 0000000180006938     libgetcaps002.obj
 0002:00000948       ??_C@_0CB@IAKPDOIC@?$CD?5?5?5verified?5assertion?5is?5FALSE@ 0000000180006948     libgetcaps002.obj
 0002:00000970       ??_C@_0CO@LGONDEPD@stdout?3?5fflush?5failed?5?9?5err?$DN?$CFd?5@ 0000000180006970     libgetcaps002.obj
 0002:000009a0       ??_C@_0CO@KBGKJPBD@stderr?3?5fflush?5failed?5?9?5err?$DN?$CFd?5@ 00000001800069a0     libgetcaps002.obj
 0002:000009d0       ??_C@_01EEMJAFIK@?6@       00000001800069d0     libgetcaps002.obj
 0002:000009d8       ??_C@_0BB@JCNMKLLK@JVMTI_ERROR_NONE@ 00000001800069d8     libgetcaps002.obj
 0002:000009f0       ??_C@_0BL@LDIMKLPH@JVMTI_ERROR_INVALID_THREAD@ 00000001800069f0     libgetcaps002.obj
 0002:00000a10       ??_C@_0CB@PJFPAIKJ@JVMTI_ERROR_INVALID_THREAD_GROU@ 0000000180006a10     libgetcaps002.obj
 0002:00000a38       ??_C@_0BN@LLMKHMNF@JVMTI_ERROR_INVALID_PRIORITY@ 0000000180006a38     libgetcaps002.obj
 0002:00000a58       ??_C@_0CB@MBOFKAGB@JVMTI_ERROR_THREAD_NOT_SUSPENDE@ 0000000180006a58     libgetcaps002.obj
 0002:00000a80       ??_C@_0BN@FABOLPBI@JVMTI_ERROR_THREAD_SUSPENDED@ 0000000180006a80     libgetcaps002.obj
 0002:00000aa0       ??_C@_0BN@FDGNOBJM@JVMTI_ERROR_THREAD_NOT_ALIVE@ 0000000180006aa0     libgetcaps002.obj
 0002:00000ac0       ??_C@_0BL@GOBIFKNJ@JVMTI_ERROR_INVALID_OBJECT@ 0000000180006ac0     libgetcaps002.obj
 0002:00000ae0       ??_C@_0BK@FCMAJPPC@JVMTI_ERROR_INVALID_CLASS@ 0000000180006ae0     libgetcaps002.obj
 0002:00000b00       ??_C@_0BP@IKLLBKEB@JVMTI_ERROR_CLASS_NOT_PREPARED@ 0000000180006b00     libgetcaps002.obj
 0002:00000b20       ??_C@_0BN@KLPPLKG@JVMTI_ERROR_INVALID_METHODID@ 0000000180006b20     libgetcaps002.obj
 0002:00000b40       ??_C@_0BN@BCEKOKND@JVMTI_ERROR_INVALID_LOCATION@ 0000000180006b40     libgetcaps002.obj
 0002:00000b60       ??_C@_0BM@DFDGPME@JVMTI_ERROR_INVALID_FIELDID@ 0000000180006b60     libgetcaps002.obj
 0002:00000b80       ??_C@_0BL@NELIEPEC@JVMTI_ERROR_NO_MORE_FRAMES@ 0000000180006b80     libgetcaps002.obj
 0002:00000ba0       ??_C@_0BJ@BDBECFDM@JVMTI_ERROR_OPAQUE_FRAME@ 0000000180006ba0     libgetcaps002.obj
 0002:00000bc0       ??_C@_0BK@MIIFNLOB@JVMTI_ERROR_TYPE_MISMATCH@ 0000000180006bc0     libgetcaps002.obj
 0002:00000be0       ??_C@_0BJ@HPCAOILC@JVMTI_ERROR_INVALID_SLOT@ 0000000180006be0     libgetcaps002.obj
 0002:00000c00       ??_C@_0BG@CHILOPNI@JVMTI_ERROR_DUPLICATE@ 0000000180006c00     libgetcaps002.obj
 0002:00000c18       ??_C@_0BG@DIEMLHKM@JVMTI_ERROR_NOT_FOUND@ 0000000180006c18     libgetcaps002.obj
 0002:00000c30       ??_C@_0BM@NHMCKHOB@JVMTI_ERROR_INVALID_MONITOR@ 0000000180006c30     libgetcaps002.obj
 0002:00000c50       ??_C@_0BO@PPEDAJGL@JVMTI_ERROR_NOT_MONITOR_OWNER@ 0000000180006c50     libgetcaps002.obj
 0002:00000c70       ??_C@_0BG@FCAIPEID@JVMTI_ERROR_INTERRUPT@ 0000000180006c70     libgetcaps002.obj
 0002:00000c88       ??_C@_0CB@EGDBNKOI@JVMTI_ERROR_INVALID_CLASS_FORMA@ 0000000180006c88     libgetcaps002.obj
 0002:00000cb0       ??_C@_0CG@DGKOGIAL@JVMTI_ERROR_CIRCULAR_CLASS_DEFI@ 0000000180006cb0     libgetcaps002.obj
 0002:00000cd8       ??_C@_0BP@ICEALPKC@JVMTI_ERROR_FAILS_VERIFICATION@ 0000000180006cd8     libgetcaps002.obj
 0002:00000cf8       ??_C@_0DC@JDACLMIO@JVMTI_ERROR_UNSUPPORTED_REDEFIN@ 0000000180006cf8     libgetcaps002.obj
 0002:00000d30       ??_C@_0DE@GKDKNOMJ@JVMTI_ERROR_UNSUPPORTED_REDEFIN@ 0000000180006d30     libgetcaps002.obj
 0002:00000d68       ??_C@_0BO@LAFKIOG@JVMTI_ERROR_INVALID_TYPESTATE@ 0000000180006d68     libgetcaps002.obj
 0002:00000d88       ??_C@_0DH@INDGCLLB@JVMTI_ERROR_UNSUPPORTED_REDEFIN@ 0000000180006d88     libgetcaps002.obj
 0002:00000dc0       ??_C@_0DE@NHEOMMGI@JVMTI_ERROR_UNSUPPORTED_REDEFIN@ 0000000180006dc0     libgetcaps002.obj
 0002:00000df8       ??_C@_0CA@EKPNJOEP@JVMTI_ERROR_UNSUPPORTED_VERSION@ 0000000180006df8     libgetcaps002.obj
 0002:00000e18       ??_C@_0BN@OFFMAHHL@JVMTI_ERROR_NAMES_DONT_MATCH@ 0000000180006e18     libgetcaps002.obj
 0002:00000e38       ??_C@_0DN@HHBBLAKE@JVMTI_ERROR_UNSUPPORTED_REDEFIN@ 0000000180006e38     libgetcaps002.obj
 0002:00000e78       ??_C@_0DO@HMBGBGNA@JVMTI_ERROR_UNSUPPORTED_REDEFIN@ 0000000180006e78     libgetcaps002.obj
 0002:00000eb8       ??_C@_0BP@PBECGKHJ@JVMTI_ERROR_UNMODIFIABLE_CLASS@ 0000000180006eb8     libgetcaps002.obj
 0002:00000ed8       ??_C@_0BK@CANILEHF@JVMTI_ERROR_NOT_AVAILABLE@ 0000000180006ed8     libgetcaps002.obj
 0002:00000ef8       ??_C@_0CE@INJKMEFK@JVMTI_ERROR_MUST_POSSESS_CAPABI@ 0000000180006ef8     libgetcaps002.obj
 0002:00000f20       ??_C@_0BJ@LBFPFPDM@JVMTI_ERROR_NULL_POINTER@ 0000000180006f20     libgetcaps002.obj
 0002:00000f40       ??_C@_0BP@CHJPNNEM@JVMTI_ERROR_ABSENT_INFORMATION@ 0000000180006f40     libgetcaps002.obj
 0002:00000f60       ??_C@_0BP@OMFMNLC@JVMTI_ERROR_INVALID_EVENT_TYPE@ 0000000180006f60     libgetcaps002.obj
 0002:00000f80       ??_C@_0BN@BIBNPHHO@JVMTI_ERROR_ILLEGAL_ARGUMENT@ 0000000180006f80     libgetcaps002.obj
 0002:00000fa0       ??_C@_0BK@KKNDHDCE@JVMTI_ERROR_NATIVE_METHOD@ 0000000180006fa0     libgetcaps002.obj
 0002:00000fc0       ??_C@_0BK@PMKCFHAE@JVMTI_ERROR_OUT_OF_MEMORY@ 0000000180006fc0     libgetcaps002.obj
 0002:00000fe0       ??_C@_0BK@NNJBDMNB@JVMTI_ERROR_ACCESS_DENIED@ 0000000180006fe0     libgetcaps002.obj
 0002:00001000       ??_C@_0BI@GHECLMNC@JVMTI_ERROR_WRONG_PHASE@ 0000000180007000     libgetcaps002.obj
 0002:00001018       ??_C@_0BF@OLIHJOII@JVMTI_ERROR_INTERNAL@ 0000000180007018     libgetcaps002.obj
 0002:00001030       ??_C@_0BO@EOHGKJHI@JVMTI_ERROR_UNATTACHED_THREAD@ 0000000180007030     libgetcaps002.obj
 0002:00001050       ??_C@_0CA@LKHFDACL@JVMTI_ERROR_INVALID_ENVIRONMENT@ 0000000180007050     libgetcaps002.obj
 0002:00001070       ??_C@_0BA@MMFHLOKK@?$DMunknown?5error?$DO@ 0000000180007070     libgetcaps002.obj
 0002:00001080       ??_C@_0CF@CBHOKDB@throwable?5?$DN?5jni?9?$DOExceptionOccur@ 0000000180007080     libgetcaps002.obj
 0002:000010a8       ??_C@_03OFAPEBGM@?$CFs?6@  00000001800070a8     libgetcaps002.obj
 0002:000010b0       ??_C@_0DM@LPIGEGNJ@s?2test?2hotspot?2jtreg?2vmTestbase@ 00000001800070b0     libgetcaps002.obj
 0002:000010f0       ??_C@_0CC@NFCNPEPK@Exception?5in?5JNI?5call?5?$CIcleared?$CJ@ 00000001800070f0     libgetcaps002.obj
 0002:00001118       ??_C@_0BJ@IBAKFIKF@jni?9?$DOExceptionDescribe?$CI?$CJ@ 0000000180007118     libgetcaps002.obj
 0002:00001138       ??_C@_0BG@GGKALKMH@jni?9?$DOExceptionClear?$CI?$CJ@ 0000000180007138     libgetcaps002.obj
 0002:00001150       ??_C@_0CF@JMGFGJLJ@?$CD?5?5?5verified?5JNI?5assertion?5is?5F@ 0000000180007150     libgetcaps002.obj
 0002:00001178       ??_C@_07KBAMPNJK@verbose@  0000000180007178     libgetcaps002.obj
 0002:00001180       ??_C@_0DN@PKJBOLAP@nsk_jvmti_parseOptions?$CI?$CJ?3?5unexp@ 0000000180007180     libgetcaps002.obj
 0002:000011c0       ??_C@_05IMBNNINJ@trace@    00000001800071c0     libgetcaps002.obj
 0002:000011c8       ??_C@_0DD@BJKGNDMB@nsk_jvmti_parseOptions?$CI?$CJ?3?5no?5va@ 00000001800071c8     libgetcaps002.obj
 0002:000011fc       ??_C@_04CGFJFPFD@none@     00000001800071fc     libgetcaps002.obj
 0002:00001204       ??_C@_06BMELKFMA@before@   0000000180007204     libgetcaps002.obj
 0002:0000120c       ??_C@_05CMKPCFDK@after@    000000018000720c     libgetcaps002.obj
 0002:00001214       ??_C@_03NFKEKGGK@all@      0000000180007214     libgetcaps002.obj
 0002:00001218       ??_C@_0DM@NDNJGJKE@nsk_jvmti_parseOptions?$CI?$CJ?3?5uexpe@ 0000000180007218     libgetcaps002.obj
 0002:00001258       ??_C@_08NBBJKJO@waittime@  0000000180007258     libgetcaps002.obj
 0002:00001268       ??_C@_0DO@CMHGAOHC@nsk_jvmti_parseOptions?$CI?$CJ?3?5not?5i@ 0000000180007268     libgetcaps002.obj
 0002:000012a8       ??_C@_0DL@LNMPBDLN@nsk_jvmti_parseOptions?$CI?$CJ?3?5negat@ 00000001800072a8     libgetcaps002.obj
 0002:000012e8       ??_C@_0DA@GMFJNOJH@nsk_jvmti_parseOptions?$CI?$CJ?3?5unkno@ 00000001800072e8     libgetcaps002.obj
 0002:00001318       ??_C@_0CO@CCIAMEAN@nsk_jvmti_parseOptions?$CI?$CJ?3?5found@ 0000000180007318     libgetcaps002.obj
 0002:00001348       ??_C@_0CJ@OEGPCGDL@nsk_jvmti_parseOptions?$CI?$CJ?3?5out?5o@ 0000000180007348     libgetcaps002.obj
 0002:00001378       ??_C@_0DI@NMBHPGGF@nsk_jvmti_parseOptions?$CI?$CJ?3?5too?5m@ 0000000180007378     libgetcaps002.obj
 0002:000013b0       ??_C@_03POGCGECB@?5?0?$HO@ 00000001800073b0     libgetcaps002.obj
 0002:000013b8       ??_C@_0CB@MLNJNCLJ@?5?5jvmti?5error?3?5code?$DN?$CFd?0?5name?$DN?$CFs@ 00000001800073b8     libgetcaps002.obj
 0002:000013e0       ??_C@_0CD@OHBGDKMK@?$CD?5?5?5jvmti?5error?3?5code?$DN?$CFd?0?5name?$DN@ 00000001800073e0     libgetcaps002.obj
 0002:00001408       ??_C@_0CG@JNNCGPHB@?$CD?5?5?5error?5expected?3?5code?$DN?$CFd?0?5na@ 0000000180007408     libgetcaps002.obj
 0002:00001430       ??_C@_0EB@IMGKPCGE@?$CIstr_obj?5?$DN?5jni?9?$DONewStringUTF?$CIco@ 0000000180007430     libgetcaps002.obj
 0002:00001480       ??_C@_0EA@HFOGGBCC@s?2test?2hotspot?2jtreg?2vmTestbase@ 0000000180007480     libgetcaps002.obj
 0002:000014c0       ??_C@_05KKCIMGE@error@     00000001800074c0     libgetcaps002.obj
 0002:000014c8       ??_C@_0CJ@JACLEAA@Test?5failed?5by?5setFailStatus?$CI?$CJ?4@ 00000001800074c8     libgetcaps002.obj
 0002:000014f8       ??_C@_0BD@HGNAOMCP@agent_data_monitor@ 00000001800074f8     libgetcaps002.obj
 0002:00001510       ??_C@_0EB@OGCLGKLN@javaVM?9?$DOGetEnv?$CI?$CIvoid?5?$CK?$CK?$CJ?$CGjvmti_@ 0000000180007510     libgetcaps002.obj
 0002:00001560       ??_C@_0EA@PNBCDMOA@s?2test?2hotspot?2jtreg?2vmTestbase@ 0000000180007560     libgetcaps002.obj
 0002:000015a0       ??_C@_0CI@DDPIFBGM@init_agent_data?$CIjvmti_env?0?5?$CGage@ 00000001800075a0     libgetcaps002.obj
 0002:000015c8       ??_C@_0DI@ILAHDLMP@?$CI?$CKagentThreadProc?$CJ?$CIjvmti_env?0?5a@ 00000001800075c8     libgetcaps002.obj
 0002:00001600       ??_C@_0BD@KDBALNLB@JVMTI?5agent?5thread@ 0000000180007600     libgetcaps002.obj
 0002:00001618       ??_C@_0BB@NOKBFPFO@java?1lang?1Thread@ 0000000180007618     libgetcaps002.obj
 0002:0000162c       ??_C@_06FALKBLGB@?$DMinit?$DO@ 000000018000762c     libgetcaps002.obj
 0002:00001638       ??_C@_0BG@IKDDPPGD@?$CILjava?1lang?1String?$DL?$CJV@ 0000000180007638     libgetcaps002.obj
 0002:00001650       ??_C@_0EB@IFJBFEKC@?$CIthreadClass?5?$DN?5jni_env?9?$DOFindCla@ 0000000180007650     libgetcaps002.obj
 0002:000016a0       ??_C@_0GF@FGFIBKKL@?$CIthreadCtor?5?$DN?5jni_env?9?$DOGetMetho@ 00000001800076a0     libgetcaps002.obj
 0002:00001708       ??_C@_0DN@NCPDJLOG@?$CIthreadName?5?$DN?5jni_env?9?$DONewStrin@ 0000000180007708     libgetcaps002.obj
 0002:00001750       ??_C@_0FE@PFKODBGC@?$CIthreadObject?5?$DN?5jni_env?9?$DONewObj@ 0000000180007750     libgetcaps002.obj
 0002:000017b0       ??_C@_0ED@HOBAHHJI@?$CIthreadGlobalRef?5?$DN?5jni_env?9?$DONew@ 00000001800077b0     libgetcaps002.obj
 0002:00001800       ??_C@_0FN@HNJJAHFC@jvmti_env?9?$DORunAgentThread?$CIagent@ 0000000180007800     libgetcaps002.obj
 0002:00001860       ??_C@_0EA@MOJDNKDF@Debuggee?5status?5sync?5aborted?5be@ 0000000180007860     libgetcaps002.obj
 0002:000018a0       ??_C@_0CO@PGPGMHBJ@No?5status?5sync?5occured?5for?5time@ 00000001800078a0     libgetcaps002.obj
 0002:000018d0       ??_C@_0CL@DOEBDPKJ@Debuggee?5was?5not?5suspended?5on?5s@ 00000001800078d0     libgetcaps002.obj
 0002:00001900       ??_C@_0EA@EEOEJAEN@status?5?$DN?5syncDebuggeeStatus?$CIjni@ 0000000180007900     libgetcaps002.obj
 0002:00001940       ??_C@_0BL@JBCFNBMB@nsk_jvmti_resetAgentData?$CI?$CJ@ 0000000180007940     libgetcaps002.obj
 0002:00001960       ??_C@_0DN@NNGECJON@jvmti_env?9?$DOSetEventNotification@ 0000000180007960     libgetcaps002.obj
 0002:000019a0       ??_C@_0EL@LPBEELIP@s?2test?2hotspot?2jtreg?2vmTestbase@ 00000001800079a0     libgetcaps002.obj
 0002:000019f0       ??_C@_0CK@JDAMFDMJ@jvmti?9?$DOSetTag?$CIo?0?5tag?$CJ?5?$DN?$DN?5JVMTI_@ 00000001800079f0     libgetcaps002.obj
 0002:00001a20       ??_C@_0CC@DAMNHKNI@Can?8t?5set?5tag?5?$CFli?5for?5object?5?$CFl@ 0000000180007a20     libgetcaps002.obj
 0002:00001a48       ??_C@_0DL@HAJPNKEF@jvmti?9?$DOGetObjectHashCode?$CIo?0?5?$CGha@ 0000000180007a48     libgetcaps002.obj
 0002:00001a88       ??_C@_0BL@JFPIEOBF@Can?8t?5get?5hash?5object?5?$CFlx?6@ 0000000180007a88     libgetcaps002.obj
 0002:00001aa8       ??_C@_0BG@DICPHBKN@setTag?3?5?$CF08x?5?$DM?9?5?$CF?53li@ 0000000180007aa8     libgetcaps002.obj
 0002:00001ac0       ??_C@_0DH@FCEEBDMJ@?$CIs?5?$DN?5jni?9?$DOGetStringUTFChars?$CIsIn@ 0000000180007ac0     libgetcaps002.obj
 0002:00001af8       ??_C@_0BJ@OKKGHDCN@Can?8t?5get?5string?5at?5?$CF?$CDp?6@ 0000000180007af8     libgetcaps002.obj
 0002:00001b18       ??_C@_0BP@EKFLGGFJ@Can?8t?5get?5string?5at?5?$CF?$CDp?3?5null?6@ 0000000180007b18     libgetcaps002.obj
 0002:00001b38       ??_C@_06ICODBHCL@?5?1?1?5?$CFs@ 0000000180007b38     libgetcaps002.obj
 0002:00001b40       ??_C@_0DB@KGFPLEGO@?$CIr?5?$DN?5jvmti?9?$DOGetTag?$CIo?0?5?$CGtag?$CJ?$CJ?5?$DN?$DN@ 0000000180007b40     libgetcaps002.obj
 0002:00001b78       ??_C@_0CO@PDAGBCGJ@Can?8t?5GetTag?5for?5object?5?$CFlx?4?5Re@ 0000000180007b78     libgetcaps002.obj
 0002:00001ba8       ??_C@_0CH@HPEODOHC@TEST_BUG?3?5Max?4?5number?5of?5refs?5r@ 0000000180007ba8     libgetcaps002.obj
 0002:00001bd0       ??_C@_0DI@PHFCABIM@?$CIr?5?$DN?5jvmti?9?$DOGetTag?$CIfrom?0?5?$CGtagFr@ 0000000180007bd0     libgetcaps002.obj
 0002:00001c08       ??_C@_0DI@MDEGFNKD@TEST_BUG?3?5Can?8t?5GetTag?5for?5obje@ 0000000180007c08     libgetcaps002.obj
 0002:00001c40       ??_C@_0DE@MLELJAHM@?$CIr?5?$DN?5jvmti?9?$DOGetTag?$CIto?0?5?$CGtagTo?$CJ?$CJ@ 0000000180007c40     libgetcaps002.obj
 0002:00001c78       ??_C@_0N@ONKJJLFA@?5?5?5?5?5?5?5?5?5?5?5?5@ 0000000180007c78     libgetcaps002.obj
 0002:00001c88       ??_C@_04DIDLCABB@?5?$CF1X@ 0000000180007c88     libgetcaps002.obj
 0002:00001c90       ??_C@_0O@ICJGKGEP@?5?5?5?50x?$CF03X?4?3?5@ 0000000180007c90     libgetcaps002.obj
 0002:00001ca0       ??_C@_04ELMIFJOO@?5?$CF1d@ 0000000180007ca0     libgetcaps002.obj
 0002:00001ca8       ??_C@_0BA@CKFEMAGK@can_tag_objects@ 0000000180007ca8     libgetcaps002.obj
 0002:00001cb8       ??_C@_0P@OGMHFGAG@?5?5?5?5?$CF?940s?3?5?$CFd?6@ 0000000180007cb8     libgetcaps002.obj
 0002:00001cc8       ??_C@_0CH@DBHACMIP@can_generate_field_modification@ 0000000180007cc8     libgetcaps002.obj
 0002:00001cf0       ??_C@_0CB@HKCHEGHM@can_generate_field_access_event@ 0000000180007cf0     libgetcaps002.obj
 0002:00001d18       ??_C@_0BC@IHDALJKK@can_get_bytecodes@ 0000000180007d18     libgetcaps002.obj
 0002:00001d30       ??_C@_0BM@IGCOPBLH@can_get_synthetic_attribute@ 0000000180007d30     libgetcaps002.obj
 0002:00001d50       ??_C@_0BL@MODEIBBH@can_get_owned_monitor_info@ 0000000180007d50     libgetcaps002.obj
 0002:00001d70       ??_C@_0CC@CIOAMEJL@can_get_current_contended_monit@ 0000000180007d70     libgetcaps002.obj
 0002:00001d98       ??_C@_0BF@GDNJHBOK@can_get_monitor_info@ 0000000180007d98     libgetcaps002.obj
 0002:00001db0       ??_C@_0O@KNEGHCNJ@can_pop_frame@ 0000000180007db0     libgetcaps002.obj
 0002:00001dc0       ??_C@_0BF@JNOFJEKM@can_redefine_classes@ 0000000180007dc0     libgetcaps002.obj
 0002:00001dd8       ??_C@_0BC@NAKCKFGO@can_signal_thread@ 0000000180007dd8     libgetcaps002.obj
 0002:00001df0       ??_C@_0BJ@PNNOBFAD@can_get_source_file_name@ 0000000180007df0     libgetcaps002.obj
 0002:00001e10       ??_C@_0BF@FGNMIJCI@can_get_line_numbers@ 0000000180007e10     libgetcaps002.obj
 0002:00001e28       ??_C@_0BP@OHHPJMLF@can_get_source_debug_extension@ 0000000180007e28     libgetcaps002.obj
 0002:00001e48       ??_C@_0BL@KLDFDFFO@can_access_local_variables@ 0000000180007e48     libgetcaps002.obj
 0002:00001e68       ??_C@_0CD@FLJBDNND@can_maintain_original_method_or@ 0000000180007e68     libgetcaps002.obj
 0002:00001e90       ??_C@_0CA@DGBPOJFO@can_generate_single_step_events@ 0000000180007e90     libgetcaps002.obj
 0002:00001eb0       ??_C@_0BO@HGCFKOLB@can_generate_exception_events@ 0000000180007eb0     libgetcaps002.obj
 0002:00001ed0       ??_C@_0BO@DLOBOJCM@can_generate_frame_pop_events@ 0000000180007ed0     libgetcaps002.obj
 0002:00001ef0       ??_C@_0BP@NGLAGCEN@can_generate_breakpoint_events@ 0000000180007ef0     libgetcaps002.obj
 0002:00001f10       ??_C@_0M@IPLCMNBD@can_suspend@ 0000000180007f10     libgetcaps002.obj
 0002:00001f20       ??_C@_0CA@LKGCMCGA@can_get_current_thread_cpu_time@ 0000000180007f20     libgetcaps002.obj
 0002:00001f40       ??_C@_0BI@PCABJHOG@can_get_thread_cpu_time@ 0000000180007f40     libgetcaps002.obj
 0002:00001f58       ??_C@_0CB@BJHOBJGL@can_generate_method_entry_event@ 0000000180007f58     libgetcaps002.obj
 0002:00001f80       ??_C@_0CA@CENDHMIA@can_generate_method_exit_events@ 0000000180007f80     libgetcaps002.obj
 0002:00001fa0       ??_C@_0CD@NGKBIBAF@can_generate_all_class_hook_eve@ 0000000180007fa0     libgetcaps002.obj
 0002:00001fc8       ??_C@_0CJ@IJLILJMI@can_generate_compiled_method_lo@ 0000000180007fc8     libgetcaps002.obj
 0002:00001ff8       ??_C@_0BM@BOAILBHN@can_generate_monitor_events@ 0000000180007ff8     libgetcaps002.obj
 0002:00002018       ??_C@_0CE@LMLAGFGP@can_generate_vm_object_alloc_ev@ 0000000180008018     libgetcaps002.obj
 0002:00002040       ??_C@_0CH@BKJALIEA@can_generate_native_method_bind@ 0000000180008040     libgetcaps002.obj
 0002:00002068       ??_C@_0CH@FKJMHFKB@can_generate_garbage_collection@ 0000000180008068     libgetcaps002.obj
 0002:00002090       ??_C@_0CA@PJIHPKOH@can_generate_object_free_events@ 0000000180008090     libgetcaps002.obj
 0002:000020b0       ??_C@_0HA@NMCIANOF@GetCapabilities?$CI?$CJ?5in?5?$CFs?5returne@ 00000001800080b0     libgetcaps002.obj
 0002:00002120       ??_C@_0FE@HHFDHPDG@s?2test?2hotspot?2jtreg?2vmTestbase@ 0000000180008120     libgetcaps002.obj
 0002:00002178       ??_C@_0CJ@BGIDMOHB@GetCapabilities?$CI?$CJ?5for?5current?5J@ 0000000180008178     libgetcaps002.obj
 0002:000021a8       ??_C@_0BO@IAKFILDF@jvmti?9?$DOGetCapabilities?$CI?$CGcaps?$CJ@ 00000001800081a8     libgetcaps002.obj
 0002:000021c8       ??_C@_0BH@MAOJMMEL@Got?5raw?5capabilities?3?6@ 00000001800081c8     libgetcaps002.obj
 0002:000021e0       ??_C@_0BF@NABNAADN@Known?5capabilities?3?6@ 00000001800081e0     libgetcaps002.obj
 0002:000021f8       ??_C@_0BO@JCKAGMHK@Checking?5capabilities?5value?3?6@ 00000001800081f8     libgetcaps002.obj
 0002:00002218       ??_C@_0P@CIIHIADO@?5?5?4?4?4?5checked?6@ 0000000180008218     libgetcaps002.obj
 0002:00002228       ??_C@_0CC@HCPFMLEK@Wait?5for?5debugee?5to?5become?5read@ 0000000180008228     libgetcaps002.obj
 0002:00002250       ??_C@_0DF@BEIBJPDJ@?$DO?$DO?$DO?5Testcase?5?$CD3?3?5Check?5capabili@ 0000000180008250     libgetcaps002.obj
 0002:00002288       ??_C@_0N@POFOADDC@agent?5thread@ 0000000180008288     libgetcaps002.obj
 0002:00002298       ??_C@_0BH@HPEOJMHL@Let?5debugee?5to?5finish?6@ 0000000180008298     libgetcaps002.obj
 0002:000022b0       ??_C@_0DJ@PCEKMEAF@?$DO?$DO?$DO?5Testcase?5?$CD2?3?5Check?5capabili@ 00000001800082b0     libgetcaps002.obj
 0002:000022f0       ??_C@_0BB@ECBNOENI@VM_INIT?5callback@ 00000001800082f0     libgetcaps002.obj
 0002:00002308       ??_C@_0DK@CGOELMAF@?$DO?$DO?$DO?5Testcase?5?$CD4?3?5Check?5capabili@ 0000000180008308     libgetcaps002.obj
 0002:00002348       ??_C@_0BC@BEKPBLPI@VM_DEATH?5callback@ 0000000180008348     libgetcaps002.obj
 0002:00002360       ??_C@_0BL@OGOOPPCN@Disable?5events?3?5?$CFd?5events?6@ 0000000180008360     libgetcaps002.obj
 0002:00002380       ??_C@_0BA@DDKAOGOI@?5?5?4?4?4?5disabled?6@ 0000000180008380     libgetcaps002.obj
 0002:00002390       ??_C@_0CA@LDMJDFDO@Exit?5with?5FAIL?5exit?5status?3?5?$CFd?6@ 0000000180008390     libgetcaps002.obj
 0002:000023b0       ??_C@_0BC@PCOLJFHD@exit?$CISTATUS_FAIL?$CJ@ 00000001800083b0     libgetcaps002.obj
 0002:000023c8       ??_C@_0CA@MNKGCBCG@nsk_jvmti_parseOptions?$CIoptions?$CJ@ 00000001800083c8     libgetcaps002.obj
 0002:000023e8       ??_C@_0DN@MIAMNFPH@?$CIjvmti?5?$DN?5nsk_jvmti_createJVMTIE@ 00000001800083e8     libgetcaps002.obj
 0002:00002430       ??_C@_0EC@ODFGFOAJ@jvmti?9?$DOSetEventCallbacks?$CI?$CGevent@ 0000000180008430     libgetcaps002.obj
 0002:00002478       ??_C@_0CL@PIACJIPK@nsk_jvmti_setAgentProc?$CIagentPro@ 0000000180008478     libgetcaps002.obj
 0002:000024a8       ??_C@_0DH@PPJABLB@?$DO?$DO?$DO?5Testcase?5?$CD1?3?5Check?5capabili@ 00000001800084a8     libgetcaps002.obj
 0002:000024e0       ??_C@_0P@LKCKDJEM@Agent_OnLoad?$CI?$CJ@ 00000001800084e0     libgetcaps002.obj
 0002:000024f0       ??_C@_0BK@EKNILGAD@Enable?5events?3?5?$CFd?5events?6@ 00000001800084f0     libgetcaps002.obj
 0002:00002510       ??_C@_0P@BAMBNLJF@?5?5?4?4?4?5enabled?6@ 0000000180008510     libgetcaps002.obj
 0002:00002530       ??_C@_1EC@JIJBPKFM@?$AAa?$AAp?$AAi?$AA?9?$AAm?$AAs?$AA?9?$AAw?$AAi?$AAn?$AA?9?$AAc?$AAo?$AAr?$AAe@ 0000000180008530     MSVCRT:thread_safe_statics.obj
 0002:00002578       ??_C@_1BK@MGMFAEKH@?$AAk?$AAe?$AAr?$AAn?$AAe?$AAl?$AA3?$AA2?$AA?4?$AAd?$AAl?$AAl@ 0000000180008578     MSVCRT:thread_safe_statics.obj
 0002:00002598       ??_C@_0BJ@JEBJOJFJ@SleepConditionVariableCS@ 0000000180008598     MSVCRT:thread_safe_statics.obj
 0002:000025b8       ??_C@_0BJ@PGPPEPCC@WakeAllConditionVariable@ 00000001800085b8     MSVCRT:thread_safe_statics.obj
 0002:000025d8       _pDefaultRawDllMain        00000001800085d8     MSVCRT:dll_dllmain.obj
 0002:000025d8       _pRawDllMain               00000001800085d8     MSVCRT:dll_dllmain.obj
 0002:000025e0       __xmm@ffffffffffffffffffffffffffffffff 00000001800085e0     MSVCRT:utility.obj
 0002:000025f0       _load_config_used          00000001800085f0     MSVCRT:loadcfg.obj
 0002:00002800       _tls_used                  0000000180008800     MSVCRT:tlssup.obj
 0002:00002828       __volatile_metadata        0000000180008828     <linker-defined>
 0002:00002c00       __rtc_iaa                  0000000180008c00     MSVCRT:initsect.obj
 0002:00002c08       __rtc_izz                  0000000180008c08     MSVCRT:initsect.obj
 0002:00002c10       __rtc_taa                  0000000180008c10     MSVCRT:initsect.obj
 0002:00002c18       __rtc_tzz                  0000000180008c18     MSVCRT:initsect.obj
 0002:00002c20       _tls_start                 0000000180008c20     MSVCRT:tlssup.obj
 0002:00002c24       _Init_thread_epoch         0000000180008c24     MSVCRT:thread_safe_statics.obj
 0002:00002c28       _tls_end                   0000000180008c28     MSVCRT:tlssup.obj
 0002:00003348       __IMPORT_DESCRIPTOR_KERNEL32 0000000180009348     kernel32:KERNEL32.dll
 0002:0000335c       __IMPORT_DESCRIPTOR_VCRUNTIME140 000000018000935c     vcruntime:VCRUNTIME140.dll
 0002:00003370       __IMPORT_DESCRIPTOR_api-ms-win-crt-heap-l1-1-0 0000000180009370     ucrt:api-ms-win-crt-heap-l1-1-0.dll
 0002:00003384       __IMPORT_DESCRIPTOR_api-ms-win-crt-runtime-l1-1-0 0000000180009384     ucrt:api-ms-win-crt-runtime-l1-1-0.dll
 0002:00003398       __IMPORT_DESCRIPTOR_api-ms-win-crt-convert-l1-1-0 0000000180009398     ucrt:api-ms-win-crt-convert-l1-1-0.dll
 0002:000033ac       __IMPORT_DESCRIPTOR_api-ms-win-crt-stdio-l1-1-0 00000001800093ac     ucrt:api-ms-win-crt-stdio-l1-1-0.dll
 0002:000033c0       __IMPORT_DESCRIPTOR_api-ms-win-crt-string-l1-1-0 00000001800093c0     ucrt:api-ms-win-crt-string-l1-1-0.dll
 0002:000033d4       __NULL_IMPORT_DESCRIPTOR   00000001800093d4     kernel32:KERNEL32.dll
 0003:00000038       _Init_global_epoch         000000018000a038     MSVCRT:thread_safe_statics.obj
 0003:00000040       __security_cookie          000000018000a040     MSVCRT:gs_cookie.obj
 0003:00000048       __security_cookie_complement 000000018000a048     MSVCRT:gs_cookie.obj
 0003:00000050       __scrt_native_dllmain_reason 000000018000a050     MSVCRT:utility.obj
 0003:00000058       __isa_available            000000018000a058     MSVCRT:cpu_disp.obj
 0003:0000005c       __isa_enabled              000000018000a05c     MSVCRT:cpu_disp.obj
 0003:00000060       __memset_fast_string_threshold 000000018000a060     MSVCRT:cpu_disp.obj
 0003:00000068       __memset_nt_threshold      000000018000a068     MSVCRT:cpu_disp.obj
 0003:00000070       __scrt_ucrt_dll_is_in_use  000000018000a070     MSVCRT:ucrt_stubs.obj
 0003:00000080       g_wrongHeapCallbacks       000000018000a080     libgetcaps002.obj
 0003:00000100       g_szTagInfo                000000018000a100     libgetcaps002.obj
 0003:00002040       g_tagFlags                 000000018000c040     libgetcaps002.obj
 0003:00002428       g_refsToVerifyCnt          000000018000c428     libgetcaps002.obj
 0003:0000242c       g_fakeUserData             000000018000c42c     libgetcaps002.obj
 0003:00002430       g_tagVisitCount            000000018000c430     libgetcaps002.obj
 0003:000033d0       g_refsToVerify             000000018000d3d0     libgetcaps002.obj
 0003:0001aad0       g_userDataError            0000000180024ad0     libgetcaps002.obj
 0003:0001ac70       ?_OptionsStorage@?1??__local_stdio_printf_options@@9@4_KA 0000000180024c70     libgetcaps002.obj
 0003:0001b238       _tls_index                 0000000180025238     MSVCRT:tlssup.obj
 0003:0001b240       __scrt_current_native_startup_state 0000000180025240     MSVCRT:utility.obj
 0003:0001b248       __scrt_native_startup_lock 0000000180025248     MSVCRT:utility.obj
 0003:0001b288       __scrt_debugger_hook_flag  0000000180025288     MSVCRT:utility_desktop.obj
 0003:0001b290       ?__type_info_root_node@@3U__type_info_node@@A 0000000180025290     MSVCRT:tncleanup.obj
 0003:0001b2a0       ?_OptionsStorage@?1??__local_stdio_scanf_options@@9@4_KA 00000001800252a0     MSVCRT:default_local_stdio_options.obj
 0003:0001b2a8       __favor                    00000001800252a8     MSVCRT:cpu_disp.obj
 0003:0001b2b0       __dyn_tls_init_callback    00000001800252b0     <common>

 entry point at        0001:00003880

 Static symbols

 0000:fffd8000       .debug$S                   0000000180000000     getcaps002.exp
 0000:fffd8000       .debug$S                   0000000180000000     vcruntime:VCRUNTIME140.dll
 0000:fffd8000       .debug$S                   0000000180000000     vcruntime:VCRUNTIME140.dll
 0000:fffd8000       .debug$S                   0000000180000000     vcruntime:VCRUNTIME140.dll
 0000:fffd8000       .debug$S                   0000000180000000     vcruntime:VCRUNTIME140.dll
 0000:fffd8000       .debug$S                   0000000180000000     vcruntime:VCRUNTIME140.dll
 0000:fffd8000       .debug$S                   0000000180000000     vcruntime:VCRUNTIME140.dll
 0000:fffd8000       .debug$S                   0000000180000000     vcruntime:VCRUNTIME140.dll
 0000:fffd8000       .debug$S                   0000000180000000     ucrt:api-ms-win-crt-convert-l1-1-0.dll
 0000:fffd8000       .debug$S                   0000000180000000     ucrt:api-ms-win-crt-heap-l1-1-0.dll
 0000:fffd8000       .debug$S                   0000000180000000     ucrt:api-ms-win-crt-heap-l1-1-0.dll
 0000:fffd8000       .debug$S                   0000000180000000     ucrt:api-ms-win-crt-heap-l1-1-0.dll
 0000:fffd8000       .debug$S                   0000000180000000     ucrt:api-ms-win-crt-heap-l1-1-0.dll
 0000:fffd8000       .debug$S                   0000000180000000     ucrt:api-ms-win-crt-runtime-l1-1-0.dll
 0000:fffd8000       .debug$S                   0000000180000000     ucrt:api-ms-win-crt-runtime-l1-1-0.dll
 0000:fffd8000       .debug$S                   0000000180000000     ucrt:api-ms-win-crt-runtime-l1-1-0.dll
 0000:fffd8000       .debug$S                   0000000180000000     ucrt:api-ms-win-crt-runtime-l1-1-0.dll
 0000:fffd8000       .debug$S                   0000000180000000     ucrt:api-ms-win-crt-runtime-l1-1-0.dll
 0000:fffd8000       .debug$S                   0000000180000000     ucrt:api-ms-win-crt-runtime-l1-1-0.dll
 0000:fffd8000       .debug$S                   0000000180000000     ucrt:api-ms-win-crt-runtime-l1-1-0.dll
 0000:fffd8000       .debug$S                   0000000180000000     ucrt:api-ms-win-crt-runtime-l1-1-0.dll
 0000:fffd8000       .debug$S                   0000000180000000     ucrt:api-ms-win-crt-runtime-l1-1-0.dll
 0000:fffd8000       .debug$S                   0000000180000000     ucrt:api-ms-win-crt-runtime-l1-1-0.dll
 0000:fffd8000       .debug$S                   0000000180000000     ucrt:api-ms-win-crt-runtime-l1-1-0.dll
 0000:fffd8000       .debug$S                   0000000180000000     ucrt:api-ms-win-crt-runtime-l1-1-0.dll
 0000:fffd8000       .debug$S                   0000000180000000     ucrt:api-ms-win-crt-runtime-l1-1-0.dll
 0000:fffd8000       .debug$S                   0000000180000000     ucrt:api-ms-win-crt-runtime-l1-1-0.dll
 0000:fffd8000       .debug$S                   0000000180000000     ucrt:api-ms-win-crt-runtime-l1-1-0.dll
 0000:fffd8000       .debug$S                   0000000180000000     ucrt:api-ms-win-crt-runtime-l1-1-0.dll
 0000:fffd8000       .debug$S                   0000000180000000     ucrt:api-ms-win-crt-stdio-l1-1-0.dll
 0000:fffd8000       .debug$S                   0000000180000000     ucrt:api-ms-win-crt-stdio-l1-1-0.dll
 0000:fffd8000       .debug$S                   0000000180000000     ucrt:api-ms-win-crt-stdio-l1-1-0.dll
 0000:fffd8000       .debug$S                   0000000180000000     ucrt:api-ms-win-crt-stdio-l1-1-0.dll
 0000:fffd8000       .debug$S                   0000000180000000     ucrt:api-ms-win-crt-stdio-l1-1-0.dll
 0000:fffd8000       .debug$S                   0000000180000000     ucrt:api-ms-win-crt-stdio-l1-1-0.dll
 0000:fffd8000       .debug$S                   0000000180000000     ucrt:api-ms-win-crt-stdio-l1-1-0.dll
 0000:fffd8000       .debug$S                   0000000180000000     ucrt:api-ms-win-crt-stdio-l1-1-0.dll
 0000:fffd8000       .debug$S                   0000000180000000     ucrt:api-ms-win-crt-stdio-l1-1-0.dll
 0000:fffd8000       .debug$S                   0000000180000000     ucrt:api-ms-win-crt-stdio-l1-1-0.dll
 0000:fffd8000       .debug$S                   0000000180000000     ucrt:api-ms-win-crt-string-l1-1-0.dll
 0000:fffd8000       .debug$S                   0000000180000000     ucrt:api-ms-win-crt-string-l1-1-0.dll
 0000:fffd8000       .debug$S                   0000000180000000     ucrt:api-ms-win-crt-string-l1-1-0.dll
 0000:fffd8000       .debug$S                   0000000180000000     ucrt:api-ms-win-crt-string-l1-1-0.dll
 0000:fffd8000       .debug$S                   0000000180000000     ucrt:api-ms-win-crt-string-l1-1-0.dll
 0000:fffd8000       .debug$S                   0000000180000000     ucrt:api-ms-win-crt-string-l1-1-0.dll
 0000:fffd8000       .debug$S                   0000000180000000     ucrt:api-ms-win-crt-string-l1-1-0.dll
 0000:fffd8000       .debug$S                   0000000180000000     ucrt:api-ms-win-crt-string-l1-1-0.dll
 0000:fffd8000       .debug$S                   0000000180000000     kernel32:KERNEL32.dll
 0000:fffd8000       .debug$S                   0000000180000000     kernel32:KERNEL32.dll
 0000:fffd8000       .debug$S                   0000000180000000     kernel32:KERNEL32.dll
 0000:fffd8000       .debug$S                   0000000180000000     kernel32:KERNEL32.dll
 0000:fffd8000       .debug$S                   0000000180000000     kernel32:KERNEL32.dll
 0000:fffd8000       .debug$S                   0000000180000000     kernel32:KERNEL32.dll
 0000:fffd8000       .debug$S                   0000000180000000     kernel32:KERNEL32.dll
 0000:fffd8000       .debug$S                   0000000180000000     kernel32:KERNEL32.dll
 0000:fffd8000       .debug$S                   0000000180000000     kernel32:KERNEL32.dll
 0000:fffd8000       .debug$S                   0000000180000000     kernel32:KERNEL32.dll
 0000:fffd8000       .debug$S                   0000000180000000     kernel32:KERNEL32.dll
 0000:fffd8000       .debug$S                   0000000180000000     kernel32:KERNEL32.dll
 0000:fffd8000       .debug$S                   0000000180000000     kernel32:KERNEL32.dll
 0000:fffd8000       .debug$S                   0000000180000000     kernel32:KERNEL32.dll
 0000:fffd8000       .debug$S                   0000000180000000     kernel32:KERNEL32.dll
 0000:fffd8000       .debug$S                   0000000180000000     kernel32:KERNEL32.dll
 0000:fffd8000       .debug$S                   0000000180000000     kernel32:KERNEL32.dll
 0000:fffd8000       .debug$S                   0000000180000000     kernel32:KERNEL32.dll
 0000:fffd8000       .debug$S                   0000000180000000     kernel32:KERNEL32.dll
 0000:fffd8000       .debug$S                   0000000180000000     kernel32:KERNEL32.dll
 0000:fffd8000       .debug$S                   0000000180000000     kernel32:KERNEL32.dll
 0000:fffd8000       .debug$S                   0000000180000000     kernel32:KERNEL32.dll
 0000:fffd8000       .debug$S                   0000000180000000     kernel32:KERNEL32.dll
 0000:fffd8000       .debug$S                   0000000180000000     kernel32:KERNEL32.dll
 0000:fffd8000       .debug$S                   0000000180000000     kernel32:KERNEL32.dll
 0000:fffd8000       .debug$S                   0000000180000000     kernel32:KERNEL32.dll
 0000:fffd8000       .debug$S                   0000000180000000     kernel32:KERNEL32.dll
 0000:fffd8000       .debug$S                   0000000180000000     kernel32:KERNEL32.dll
 0001:00000ee4       addRefToVerify             0000000180001ee4 f   libgetcaps002.obj
 0001:00000f50       agentProc                  0000000180001f50 f   libgetcaps002.obj
 0001:00000fd8       agentThreadWrapper         0000000180001fd8 f   libgetcaps002.obj
 0001:0000125c       checkCapabilities          000000018000225c f   libgetcaps002.obj
 0001:000013b0       checkCapabilitiesValue     00000001800023b0 f   libgetcaps002.obj
 0001:00001a84       check_option               0000000180002a84 f   libgetcaps002.obj
 0001:00001ccc       file_basename              0000000180002ccc f   libgetcaps002.obj
 0001:00002914       printKnownCapabilities     0000000180003914 f   libgetcaps002.obj
 0001:00002c54       printRawCapabilities       0000000180003c54 f   libgetcaps002.obj
 0001:00002d64       startAgentThreadWrapper    0000000180003d64 f   libgetcaps002.obj
 0001:000030a4       syncDebuggeeStatus         00000001800040a4 f   libgetcaps002.obj
 0001:00003344       capture_previous_context   0000000180004344 f   MSVCRT:gs_report.obj
 0001:000033b8       ?__scrt_initialize_thread_safe_statics@@YAHXZ 00000001800043b8 f   MSVCRT:thread_safe_statics.obj
 0001:00003488       ?__scrt_uninitialize_thread_safe_statics@@YAXXZ 0000000180004488 f   MSVCRT:thread_safe_statics.obj
 0001:00003530       $$000000                   0000000180004530     MSVCRT:amdsecgs.obj
 0001:00003560       ?dllmain_crt_dispatch@@YAHQEAUHINSTANCE__@@KQEAX@Z 0000000180004560 f   MSVCRT:dll_dllmain.obj
 0001:000035b0       ?dllmain_crt_process_attach@@YAHQEAUHINSTANCE__@@QEAX@Z 00000001800045b0 f   MSVCRT:dll_dllmain.obj
 0001:000036c8       ?dllmain_crt_process_detach@@YAH_N@Z 00000001800046c8 f   MSVCRT:dll_dllmain.obj
 0001:0000374c       ?dllmain_dispatch@@YAHQEAUHINSTANCE__@@KQEAX@Z 000000018000474c f   MSVCRT:dll_dllmain.obj
 0001:00004160       $$000000                   0000000180005160     MSVCRT:guard_dispatch.obj
 0001:00004180       $$000000                   0000000180005180     MSVCRT:guard_xfg_dispatch.obj
 0001:00004196       ?fin$0@?0??dllmain_crt_process_attach@@YAHQEAUHINSTANCE__@@QEAX@Z@4HA 0000000180005196 f   MSVCRT:dll_dllmain.obj
 0001:000041ad       ?fin$0@?0??dllmain_crt_process_detach@@YAH_N@Z@4HA 00000001800051ad f   MSVCRT:dll_dllmain.obj
 0001:000041c6       ?fin$1@?0??dllmain_crt_process_detach@@YAH_N@Z@4HA 00000001800051c6 f   MSVCRT:dll_dllmain.obj
 0001:000041da       ?filt$0@?0??dllmain_dispatch@@YAHQEAUHINSTANCE__@@KQEAX@Z@4HA 00000001800051da f   MSVCRT:dll_dllmain.obj
 0001:00004210       __scrt_is_nonwritable_in_current_image$filt$0 0000000180005210 f   MSVCRT:utility.obj
 0002:00000218       ?__scrt_initialize_tss_var@@3P6AHXZEA 0000000180006218     MSVCRT:thread_safe_statics.obj
 0002:00000340       ?opcLengths@@3QBEB         0000000180006340     libgetcaps002.obj
 0002:00002520       GS_ExceptionPointers       0000000180008520     MSVCRT:gs_report.obj
 0002:00002c30       $unwind$fprintf            0000000180008c30     libgetcaps002.obj
 0002:00002c3c       $unwind$printf             0000000180008c3c     libgetcaps002.obj
 0002:00002c48       $unwind$?NewObject@JNIEnv_@@QEAAPEAV_jobject@@PEAV_jclass@@PEAU_jmethodID@@ZZ 0000000180008c48     libgetcaps002.obj
 0002:00002c48       $unwind$nsk_lcomplain      0000000180008c48     libgetcaps002.obj
 0002:00002c48       $unwind$nsk_ldisplay       0000000180008c48     libgetcaps002.obj
 0002:00002c50       $unwind$nsk_jvmti_waitForSync 0000000180008c50     libgetcaps002.obj
 0002:00002c50       $unwind$nsk_lvdisplay      0000000180008c50     libgetcaps002.obj
 0002:00002c50       $unwind$_RTC_Initialize    0000000180008c50     MSVCRT:initsect.obj
 0002:00002c50       $unwind$_RTC_Terminate     0000000180008c50     MSVCRT:initsect.obj
 0002:00002c50       $unwind$?__scrt_initialize_thread_safe_statics@@YAHXZ 0000000180008c50     MSVCRT:thread_safe_statics.obj
 0002:00002c5c       $unwind$nsk_complain       0000000180008c5c     libgetcaps002.obj
 0002:00002c5c       $unwind$nsk_printf         0000000180008c5c     libgetcaps002.obj
 0002:00002c64       $unwind$nsk_lvcomplain     0000000180008c64     libgetcaps002.obj
 0002:00002c7c       $unwind$nsk_ltrace         0000000180008c7c     libgetcaps002.obj
 0002:00002c7c       $unwind$__report_gsfailure 0000000180008c7c     MSVCRT:gs_report.obj
 0002:00002c84       $unwind$agentProc          0000000180008c84     libgetcaps002.obj
 0002:00002c84       $unwind$callbackVMInit     0000000180008c84     libgetcaps002.obj
 0002:00002c84       $unwind$nsk_lvtrace        0000000180008c84     libgetcaps002.obj
 0002:00002c84       $unwind$__raise_securityfailure 0000000180008c84     MSVCRT:gs_report.obj
 0002:00002c84       $unwind$__scrt_initialize_crt 0000000180008c84     MSVCRT:utility.obj
 0002:00002c84       $unwind$__scrt_initialize_onexit_tables 0000000180008c84     MSVCRT:utility.obj
 0002:00002c84       $unwind$__scrt_release_startup_lock 0000000180008c84     MSVCRT:utility.obj
 0002:00002c84       $unwind$__scrt_uninitialize_crt 0000000180008c84     MSVCRT:utility.obj
 0002:00002c84       $unwind$_onexit            0000000180008c84     MSVCRT:utility.obj
 0002:00002c8c       $unwind$nsk_lverify        0000000180008c8c     libgetcaps002.obj
 0002:00002c9c       $unwind$nsk_vprintf        0000000180008c9c     libgetcaps002.obj
 0002:00002cac       $unwind$?nsk_jni_lverify@@YAHHPEAUJNIEnv_@@HQEBDH1ZZ 0000000180008cac     libgetcaps002.obj
 0002:00002cc0       $unwind$?nsk_jni_check_exception@@YAHPEAUJNIEnv_@@QEBDH@Z 0000000180008cc0     libgetcaps002.obj
 0002:00002cdc       $unwind$nsk_jvmti_parseOptions 0000000180008cdc     libgetcaps002.obj
 0002:00002cf8       $unwind$nsk_jvmti_createJVMTIEnv 0000000180008cf8     libgetcaps002.obj
 0002:00002d0c       $unwind$Java_nsk_jvmti_unit_FollowReferences_FollowRefObjects_resetTags 0000000180008d0c     libgetcaps002.obj
 0002:00002d0c       $unwind$addRefToVerify     0000000180008d0c     libgetcaps002.obj
 0002:00002d0c       $unwind$nsk_jvmti_resetAgentData 0000000180008d0c     libgetcaps002.obj
 0002:00002d0c       $unwind$nsk_jvmti_resumeSync 0000000180008d0c     libgetcaps002.obj
 0002:00002d0c       $unwind$nsk_jvmti_setFailStatus 0000000180008d0c     libgetcaps002.obj
 0002:00002d0c       $unwind$__scrt_initialize_default_local_stdio_options 0000000180008d0c     MSVCRT:default_local_stdio_options.obj
 0002:00002d0c       $unwind$?dllmain_crt_dispatch@@YAHQEAUHINSTANCE__@@KQEAX@Z 0000000180008d0c     MSVCRT:dll_dllmain.obj
 0002:00002d0c       $unwind$DllMain            0000000180008d0c     MSVCRT:dll_dllmain_stub.obj
 0002:00002d0c       $unwind$__GSHandlerCheck   0000000180008d0c     MSVCRT:gshandler.obj
 0002:00002d0c       $unwind$?__scrt_uninitialize_thread_safe_statics@@YAXXZ 0000000180008d0c     MSVCRT:thread_safe_statics.obj
 0002:00002d0c       $unwind$__scrt_acquire_startup_lock 0000000180008d0c     MSVCRT:utility.obj
 0002:00002d0c       $unwind$__scrt_dllmain_after_initialize_c 0000000180008d0c     MSVCRT:utility.obj
 0002:00002d0c       $unwind$__scrt_dllmain_before_initialize_c 0000000180008d0c     MSVCRT:utility.obj
 0002:00002d0c       $unwind$__scrt_dllmain_crt_thread_attach 0000000180008d0c     MSVCRT:utility.obj
 0002:00002d0c       $unwind$__scrt_dllmain_crt_thread_detach 0000000180008d0c     MSVCRT:utility.obj
 0002:00002d0c       $unwind$__scrt_dllmain_uninitialize_c 0000000180008d0c     MSVCRT:utility.obj
 0002:00002d0c       $unwind$__scrt_dllmain_uninitialize_critical 0000000180008d0c     MSVCRT:utility.obj
 0002:00002d0c       $unwind$atexit             0000000180008d0c     MSVCRT:utility.obj
 0002:00002d14       $unwind$nsk_jvmti_enableEvents 0000000180008d14     libgetcaps002.obj
 0002:00002d2c       $unwind$nsk_jvmti_lverify  0000000180008d2c     libgetcaps002.obj
 0002:00002d40       $unwind$exitOnError        0000000180008d40     libgetcaps002.obj
 0002:00002d50       $unwind$check_option       0000000180008d50     libgetcaps002.obj
 0002:00002d50       $unwind$printKnownCapabilities 0000000180008d50     libgetcaps002.obj
 0002:00002d50       $unwind$_DllMainCRTStartup 0000000180008d50     MSVCRT:dll_dllmain.obj
 0002:00002d60       $unwind$Java_nsk_share_jvmti_ArgumentHandler_getAgentOptionsString 0000000180008d60     libgetcaps002.obj
 0002:00002d74       $unwind$Java_nsk_jvmti_unit_FollowReferences_FollowRefObjects_getTag 0000000180008d74     libgetcaps002.obj
 0002:00002d74       $unwind$Java_nsk_share_jvmti_DebugeeClass_checkStatus 0000000180008d74     libgetcaps002.obj
 0002:00002d74       $unwind$agentThreadWrapper 0000000180008d74     libgetcaps002.obj
 0002:00002d84       $unwind$startAgentThreadWrapper 0000000180008d84     libgetcaps002.obj
 0002:00002da0       $unwind$syncDebuggeeStatus 0000000180008da0     libgetcaps002.obj
 0002:00002da0       $unwind$__scrt_dllmain_exception_filter 0000000180008da0     MSVCRT:utility.obj
 0002:00002db4       $unwind$Java_nsk_share_jvmti_DebugeeClass_resetAgentData 0000000180008db4     libgetcaps002.obj
 0002:00002dbc       $unwind$MA_checkStatus     0000000180008dbc     libgetcaps002.obj
 0002:00002dd0       $unwind$Java_nsk_jvmti_unit_FollowReferences_FollowRefObjects_setTag 0000000180008dd0     libgetcaps002.obj
 0002:00002de8       $unwind$Java_nsk_jvmti_unit_FollowReferences_FollowRefObjects_addRefToVerify 0000000180008de8     libgetcaps002.obj
 0002:00002de8       $unwind$checkCapabilitiesValue 0000000180008de8     libgetcaps002.obj
 0002:00002e04       $unwind$Agent_Initialize   0000000180008e04     libgetcaps002.obj
 0002:00002e24       $unwind$printRawCapabilities 0000000180008e24     libgetcaps002.obj
 0002:00002e3c       $unwind$checkCapabilities  0000000180008e3c     libgetcaps002.obj
 0002:00002e58       $unwind$callbackVMDeath    0000000180008e58     libgetcaps002.obj
 0002:00002e64       $unwind$capture_previous_context 0000000180008e64     MSVCRT:gs_report.obj
 0002:00002e70       $unwind$__GSHandlerCheckCommon 0000000180008e70     MSVCRT:gshandler.obj
 0002:00002e78       $xdatasym                  0000000180008e78     MSVCRT:amdsecgs.obj
 0002:00002e7c       $unwind$?dllmain_crt_process_attach@@YAHQEAUHINSTANCE__@@QEAX@Z 0000000180008e7c     MSVCRT:dll_dllmain.obj
 0002:00002eb8       $unwind$?fin$0@?0??dllmain_crt_process_attach@@YAHQEAUHINSTANCE__@@QEAX@Z@4HA 0000000180008eb8     MSVCRT:dll_dllmain.obj
 0002:00002eb8       $unwind$?fin$0@?0??dllmain_crt_process_detach@@YAH_N@Z@4HA 0000000180008eb8     MSVCRT:dll_dllmain.obj
 0002:00002eb8       $unwind$?fin$1@?0??dllmain_crt_process_detach@@YAH_N@Z@4HA 0000000180008eb8     MSVCRT:dll_dllmain.obj
 0002:00002ec0       $unwind$?dllmain_crt_process_detach@@YAH_N@Z 0000000180008ec0     MSVCRT:dll_dllmain.obj
 0002:00002f14       $unwind$?dllmain_dispatch@@YAHQEAUHINSTANCE__@@KQEAX@Z 0000000180008f14     MSVCRT:dll_dllmain.obj
 0002:00002f3c       $unwind$?filt$0@?0??dllmain_dispatch@@YAHQEAUHINSTANCE__@@KQEAX@Z@4HA 0000000180008f3c     MSVCRT:dll_dllmain.obj
 0002:00002f44       $unwind$__scrt_is_nonwritable_in_current_image 0000000180008f44     MSVCRT:utility.obj
 0002:00002f64       $unwind$__scrt_is_nonwritable_in_current_image$filt$0 0000000180008f64     MSVCRT:utility.obj
 0002:00002f6c       $unwind$__scrt_fastfail    0000000180008f6c     MSVCRT:utility_desktop.obj
 0002:00002f7c       $unwind$__security_init_cookie 0000000180008f7c     MSVCRT:gs_support.obj
 0002:00002f88       $unwind$__isa_available_init 0000000180008f88     MSVCRT:cpu_disp.obj
 0002:00002f98       $xdatasym                  0000000180008f98     MSVCRT:guard_dispatch.obj
 0002:00002fa0       $xdatasym                  0000000180008fa0     MSVCRT:guard_xfg_dispatch.obj
 0002:00002fb0       .edata                     0000000180008fb0     getcaps002.exp
 0002:00002fd8       rgpv                       0000000180008fd8     getcaps002.exp
 0002:00003018       rgszName                   0000000180009018     getcaps002.exp
 0002:00003058       rgwOrd                     0000000180009058     getcaps002.exp
 0002:00003078       szName                     0000000180009078     getcaps002.exp
 0002:00003087       $N00001                    0000000180009087     getcaps002.exp
 0002:00003096       $N00002                    0000000180009096     getcaps002.exp
 0002:000030a3       $N00003                    00000001800090a3     getcaps002.exp
 0002:000030e8       $N00004                    00000001800090e8     getcaps002.exp
 0002:00003125       $N00005                    0000000180009125     getcaps002.exp
 0002:0000316d       $N00006                    000000018000916d     getcaps002.exp
 0002:000031ad       $N00007                    00000001800091ad     getcaps002.exp
 0002:000031ea       $N00008                    00000001800091ea     getcaps002.exp
 0002:00003225       $N00009                    0000000180009225     getcaps002.exp
 0002:00003253       $N00010                    0000000180009253     getcaps002.exp
 0002:00003284       $N00011                    0000000180009284     getcaps002.exp
 0002:000032b3       $N00012                    00000001800092b3     getcaps002.exp
 0002:000032e2       $N00013                    00000001800092e2     getcaps002.exp
 0002:00003317       $N00014                    0000000180009317     getcaps002.exp
 0002:00003326       $N00015                    0000000180009326     getcaps002.exp
 0002:00003336       $N00016                    0000000180009336     getcaps002.exp
 0002:0000379a       .idata$6                   000000018000979a     kernel32:KERNEL32.dll
 0002:000037fe       .idata$6                   00000001800097fe     vcruntime:VCRUNTIME140.dll
 0002:00003990       .idata$6                   0000000180009990     ucrt:api-ms-win-crt-heap-l1-1-0.dll
 0002:000039b0       .idata$6                   00000001800099b0     ucrt:api-ms-win-crt-runtime-l1-1-0.dll
 0002:000039d2       .idata$6                   00000001800099d2     ucrt:api-ms-win-crt-convert-l1-1-0.dll
 0002:000039f4       .idata$6                   00000001800099f4     ucrt:api-ms-win-crt-stdio-l1-1-0.dll
 0002:00003a14       .idata$6                   0000000180009a14     ucrt:api-ms-win-crt-string-l1-1-0.dll
 0003:00000000       ?codeAttributeName@@3PEBDEB 000000018000a000     libgetcaps002.obj
 0003:00000008       ?lineNumberAttributeName@@3PEBDEB 000000018000a008     libgetcaps002.obj
 0003:00000010       ?localVarAttributeName@@3PEBDEB 000000018000a010     libgetcaps002.obj
 0003:00000018       ?localVarTypeAttributeName@@3PEBDEB 000000018000a018     libgetcaps002.obj
 0003:00000020       ?stackMapAttributeName@@3PEBDEB 000000018000a020     libgetcaps002.obj
 0003:00000028       ?callBytes@@3PAEA          000000018000a028     libgetcaps002.obj
 0003:0000002c       ?allocBytes@@3PAEA         000000018000a02c     libgetcaps002.obj
 0003:00000030       events                     000000018000a030     libgetcaps002.obj
 0003:0001aad4       redefineAttempted          0000000180024ad4     libgetcaps002.obj
 0003:0001aad8       nsk_context                0000000180024ad8     libgetcaps002.obj
 0003:0001aae4       redefineSucceed            0000000180024ae4     libgetcaps002.obj
 0003:0001aae8       agentFailed                0000000180024ae8     libgetcaps002.obj
 0003:0001aaec       currentAgentStatus         0000000180024aec     libgetcaps002.obj
 0003:0001aaf0       context                    0000000180024af0     libgetcaps002.obj
 0003:0001aba8       agentThread                0000000180024ba8     libgetcaps002.obj
 0003:0001abb0       agentThreadProc            0000000180024bb0     libgetcaps002.obj
 0003:0001abb8       agentThreadArg             0000000180024bb8     libgetcaps002.obj
 0003:0001abc0       agent_data                 0000000180024bc0     libgetcaps002.obj
 0003:0001abd0       jvmti_env                  0000000180024bd0     libgetcaps002.obj
 0003:0001abd8       jvm                        0000000180024bd8     libgetcaps002.obj
 0003:0001abe0       jni_env                    0000000180024be0     libgetcaps002.obj
 0003:0001abe8       checkStatus_func           0000000180024be8     libgetcaps002.obj
 0003:0001abf0       ?codeAttributeIndex@@3GA   0000000180024bf0     libgetcaps002.obj
 0003:0001abf4       ?lineNumberAttributeIndex@@3GA 0000000180024bf4     libgetcaps002.obj
 0003:0001abf8       ?localVarAttributeIndex@@3GA 0000000180024bf8     libgetcaps002.obj
 0003:0001abfc       ?localVarTypeAttributeIndex@@3GA 0000000180024bfc     libgetcaps002.obj
 0003:0001ac00       ?stackMapAttributeIndex@@3GA 0000000180024c00     libgetcaps002.obj
 0003:0001ac04       ?stackFrameOffset@@3GA     0000000180024c04     libgetcaps002.obj
 0003:0001ac08       ?mode@@3HA                 0000000180024c08     libgetcaps002.obj
 0003:0001ac0c       ?constantPoolSize@@3GA     0000000180024c0c     libgetcaps002.obj
 0003:0001ac10       ?orig@@3PEBEEB             0000000180024c10     libgetcaps002.obj
 0003:0001ac18       ?gen@@3PEAEEA              0000000180024c18     libgetcaps002.obj
 0003:0001ac20       ?inputPos@@3PEAEEA         0000000180024c20     libgetcaps002.obj
 0003:0001ac28       ?endPos@@3PEBEEB           0000000180024c28     libgetcaps002.obj
 0003:0001ac30       ?genPos@@3PEAEEA           0000000180024c30     libgetcaps002.obj
 0003:0001ac38       ?markPos@@3PEAEEA          0000000180024c38     libgetcaps002.obj
 0003:0001ac40       ?constantPool@@3PEAPEADEA  0000000180024c40     libgetcaps002.obj
 0003:0001ac48       ?constantPoolCount@@3GA    0000000180024c48     libgetcaps002.obj
 0003:0001ac4c       ?zeroBytes@@3PAEA          0000000180024c4c     libgetcaps002.obj
 0003:0001ac50       ?codeLength@@3IA           0000000180024c50     libgetcaps002.obj
 0003:0001ac58       ?map@@3PEAIEA              0000000180024c58     libgetcaps002.obj
 0003:0001ac60       ?widening@@3PEACEA         0000000180024c60     libgetcaps002.obj
 0003:0001ac68       timeout                    0000000180024c68     libgetcaps002.obj
 0003:0001ac80       GS_ExceptionRecord         0000000180024c80     MSVCRT:gs_report.obj
 0003:0001ad20       GS_ContextRecord           0000000180024d20     MSVCRT:gs_report.obj
 0003:0001b1f0       ?g_tss_cv@@3U_RTL_CONDITION_VARIABLE@@A 00000001800251f0     MSVCRT:thread_safe_statics.obj
 0003:0001b1f8       ?g_tss_event@@3PEAXEA      00000001800251f8     MSVCRT:thread_safe_statics.obj
 0003:0001b200       ?g_tss_mutex@@3U_RTL_CRITICAL_SECTION@@A 0000000180025200     MSVCRT:thread_safe_statics.obj
 0003:0001b228       ?g_sleep_condition_variable_cs@@3P6AHPEAU_RTL_CONDITION_VARIABLE@@PEAU_RTL_CRITICAL_SECTION@@K@ZEA 0000000180025228     MSVCRT:thread_safe_statics.obj
 0003:0001b230       ?g_wake_all_condition_variable@@3P6AXPEAU_RTL_CONDITION_VARIABLE@@@ZEA 0000000180025230     MSVCRT:thread_safe_statics.obj
 0003:0001b23c       ?__proc_attached@@3HA      000000018002523c     MSVCRT:dll_dllmain.obj
 0003:0001b250       ?is_initialized_as_dll@@3_NA 0000000180025250     MSVCRT:utility.obj
 0003:0001b251       ?module_local_atexit_table_initialized@@3_NA 0000000180025251     MSVCRT:utility.obj
 0003:0001b258       ?module_local_atexit_table@@3U_onexit_table_t@@A 0000000180025258     MSVCRT:utility.obj
 0003:0001b270       ?module_local_at_quick_exit_table@@3U_onexit_table_t@@A 0000000180025270     MSVCRT:utility.obj
